:0200000480007A
:10000000B72F0000938F0F8073900F3015A8130047
:100010000000130000001300000013000000130094
:100020000000130000001300000013000000130084
:100030000000130000001300000013000000010086
:10004000970200009382020C73905230814001416C
:100050008141014281420143814301448144014580
:100060008145014681460147814701488148014950
:100070008149014A814A014B814B014C814C014D20
:10008000814D014E814E014F814F971102009381A6
:1000900021D6170502001305E556979503009385B1
:1000A000A57701461122170502001305254897057B
:1000B00002009385A5530146C52817A50300130523
:1000C000E57597B503009385257537B6ABAB130679
:1000D000B6BAD92817B1030013014174EF608059F3
:1000E000860293D21200F512638802008242110147
:1000F0006F00001073002030824211017300203025
:10010000711116C0F3222034E3CC02FC82421101AB
:10011000130141F806C20AC40EC612C816CA1ACC88
:100120001ECE22D026D22AD42ED632D836DA3ADCC7
:100130003EDEC2C0C6C2CAC4CEC6D2C8D6CADACC97
:10014000DECEE2D0E6D2EAD4EED6F2D8F6DAFADCA7
:10015000FEDE73252034F32510340A8601A07310C7
:10016000153492402241B2414242D2426243F243AC
:10017000025492542255B2554256D2566257F25703
:10018000064896482649B649464AD64A664BF64B33
:10019000065C965C265DB65D465ED65E665FF65F83
:1001A0001301C1077300203010C16374B50011053D
:1001B000E5BF828000000000000000000000000099
:1001C000000000000000000000000000000000002F
:1001D000000000000000000000000000000000001F
:1001E000000000000000000000000000000000000F
:1001F000197106C00AC20EC412C616C81ACA1ECC8D
:1002000022CE26D02AD22ED432D636D83ADA3EDCC6
:1002100042DEC6C0CAC2CEC4D2C6D6C8DACADECC96
:10022000E2CEE6D0EAD2EED4F2D6F6D8FADAFEDCA6
:100230009702020083A2C23223A02200F3221034CC
:1002400096DEEF00002B170102000321613102410D
:10025000F65273901234B72200009382028873A082
:10026000023082403242C2425243E24372448254DC
:100270001255A2553256C2565257E2577258864806
:100280001649A649364AC64A564BE64B764C865C1A
:10029000165DA65D365EC65E565FE65F0961730059
:1002A0002030970202009382E23523A0120023A29D
:1002B000220023A4320023A6420023A8520023AA2E
:1002C000620023AC720023AE820023A0920223A21C
:1002D000A20223A4B20223A6C20223A8D20223AA06
:1002E000E20223ACF20223AE020323A0120523A2F2
:1002F000220523A4320523A6420523A8520523AADA
:10030000620523AC720523AE820523A0920723A2C7
:10031000A20723A4B20723A6C20723A8D20723AAB1
:10032000E20723ACF207EF40702E17010200032111
:1003300021230241F65273901234B72200009382B7
:10034000028873A0023082403242C2425243E243EA
:10035000724482541255A2553256C2565257E25731
:10036000725886481649A649364AC64A564BE64B45
:10037000764C865C165DA65D365EC65E565FE65FB1
:10038000096173002030970202009382A22783A0A4
:10039000020003A1420083A1820003A2C20083A243
:1003A000020103A3420183A3820103A4C20183A427
:1003B000020203A5420283A5820203A6C20283A60B
:1003C000020303A7420383A7820303A8C20383A8EF
:1003D000020403A9420483A9820403AAC20483AAD3
:1003E000020503AB420583AB820503ACC20583ACB7
:1003F000020603AD420683AD820603AEC20683AE9B
:10040000020703AFC20983AF820782807370043092
:10041000197106C00AC20EC412C616C81ACA1ECC6A
:1004200022CE26D02AD22ED432D636D83ADA3EDCA4
:1004300042DEC6C0CAC2CEC4D2C6D6C8DACADECC74
:10044000E2CEE6D0EAD2EED4F2D6F6D8FADAFEDC84
:100450009702020083A2C21023A0220086DEEF20B2
:10046000E035170102000321A10F0241F6527390FB
:100470001234B72200009382028873A002308240B7
:100480003242C2425243E243724482541255A25550
:100490003256C2565257E257725886481649A649F4
:1004A000364AC64A564BE64B764C865C165DA65DD0
:1004B000365EC65E565FE65F09617300203073707A
:1004C000043001A07310453082807325403073F0F2
:1004D00043308280970700009387A7FE232EB5FE46
:1004E0002322C5FA232635F82320F5F8130505F84D
:1004F0008280411106C6EF40900EEF10D01301E547
:10050000B24041018280B24041016F20202B93070D
:1005100085007D575CC118C55CC51CC9232005003A
:1005200082802328050082805C41DCC1984798C501
:1005300098474CC38CC788C91C4185071CC1828061
:100540009041FD57130785006314F60039A83E87D4
:100550005C439443E37DD6FEDCC18CC798C54CC395
:1005600088C91C4185071CC1828018495C43EDB7CE
:10057000584114451C4914C71845544154C3D84325
:100580006314A7001845D8C32328050088437D15A8
:1005900088C382803041AE8701CE4C455841B29528
:1005A0004CC563E4E5000C414CC53E856F30B02777
:1005B0008280411122C406C62A8426C2EF20301947
:1005C0003C44635BF0025C5085CB9304440209A871
:1005D0003C44FD173CC43C446350F0025C5089CF5E
:1005E0002685EF20405F6DD5EF20207F3C44FD172E
:1005F0003CC43C44E344F0FEFD573CC4EF2070177C
:10060000EF20F0147C40635BF0021C4885CB930420
:10061000040109A87C40FD177CC07C406350F002B7
:100620001C4889CF2685EF20005B6DD5EF20E07A4E
:100630007C40FD177CC07C40E344F0FEFD577CC04D
:100640002244B240924441016F20B01229C54111A9
:1006500022C426C22A8406C6AE84EF20500F34403E
:100660005C5C1840232C0402B387F6027D5670C0F0
:1006700018C430C4B386D740BA9736975CC058C404
:1006800091EC1C489DE3EF20D00EB24022449244EE
:100690000545410182807370043001A013050401F7
:1006A000BD3513054402A535F9BF13050401EF203C
:1006B00080528547E319F5FC913BF1B701E5737072
:1006C000043001A0011126CA4AC84EC606CE22CC6B
:1006D000B2892E89AA84A5C53305B502130555052F
:1006E000EF30207C2A8435C1930745051CC144DCCA
:1006F00023202405EF20B00534405C5C18407D5673
:10070000B387F602232C040270C018C430C413054A
:100710000401B386D740BA9736975CC058C4C53B2E
:1007200013054402ED33EF20D0042308340522855D
:10073000F2406244D2444249B249056182801305C5
:100740004005EF3000762A8401E57370043001A083
:1007500000C071BF01E57370043001A06375B5007E
:100760007370043001A0411122C409462E848145D2
:1007700006C6A93711C500DDB2402244410182807E
:100780007370043001A05D7186C6A2C4A6C2CAC03F
:100790004EDE52DC56DA5AD85ED632C6630A051CE3
:1007A0006382051C89476399F600585D8547630598
:1007B000F7007370043001A03689AE842A84EF20DC
:1007C000406411E5B24781C77370043001A0EF2087
:1007D0000078185C5C5C014B894BFD59130A0401DD
:1007E000930A44026365F70C63077919B247638182
:1007F000072463150B002808EF200051EF206077D5
:10080000EF10205AEF20A0747C406394370123221C
:1008100004043C446394370123240404EF206075EE
:100820006C002808EF206050631E051EEF20207228
:10083000185C5C5C630CF70AEF20A073EF2020715A
:100840003C44634FF00039A85685EF20C03819C1E9
:10085000EF20A0583C44FD173CC43C446354F000D6
:100860005C50FDF323243405EF20A070EF20206EB0
:100870007C40634FF00039A85285EF20C03519C184
:10088000EF20A0557C40FD177CC07C406354F000F5
:100890001C48FDF323223405EF20A06DEF10607596
:1008A000054BEF20C06A185C5C5CE37FF7F23040D8
:1008B0006305060C631F09120844A685EF30A07675
:1008C0001C4434405840B6971CC463EAE70A1C5CD9
:1008D00014405850850714C41CDC5DC7130544023E
:1008E000EF20602F85476311F50AC9A8EF206068E3
:1008F000B2455285EF20E00FEF2060653C44634F26
:10090000F00039A85685EF20002D19C1EF20E04CEA
:100910003C44FD173CC43C446354F0005C50FDF380
:1009200023243405EF20E064EF2060627C40634FB5
:10093000F00039A85285EF20002A19C1EF20E049C4
:100940007C40FD177CC07C406354F0001C48FDF3E4
:1009500023223405EF20E061EF10A06931F17D34EE
:10096000054B81B73C41E38F07E27370043001A06F
:100970007370043001A0304021E61C4085C71C5C28
:10098000585085071CDC39FBEF20A05E0545B640BA
:10099000264496440649F259625AD25A425BB25BE7
:1009A000616182804840EF20E0511C5C5850232256
:1009B000040085071CDCE31307F279D5813CE9B715
:1009C0004844A685EF3020663C4058441440B307A5
:1009D000F0403E9758C4637CD7025840BA975CC435
:1009E00009475C506306E902185C050718DCC9DF9B
:1009F000F5B54844A685EF3000633C4058441440A8
:100A0000B307F0403E9758C4E37CD7FCF9B75C507D
:100A1000185C79DB185C7D1718DC185C050718DC9E
:100A2000A5D76DBD22857136EF10A05C014585B755
:100A3000EF2020540145A1BF411126C2AA8413050D
:100A4000400522C406C6EF30C0452A8415CD232CAC
:100A50000502FD577CC10547410558DC3CC42322F3
:100A60000400232004002324040023260400232060
:100A7000040423089404613C13054402493C814664
:100A800001468145228501332285B24022449244A9
:100A9000410182800DC5411122C426C206C64AC04A
:100AA000032945002A84EF2000358144630CA90006
:100AB000B2402244268502499244410182807370EB
:100AC000043001A05C448544FD175CC4F5F3814605
:100AD0000146814522854539E1BF31CDA1C90111CA
:100AE00022CC26CA4AC852C406CE4EC68947B6840E
:100AF00032892E8A2A846399F600585D8547630FF0
:100B0000F7047370043001A0C932185C5C5CAA89D8
:100B10006366F70281444E857532F2406244268551
:100B20004249D244B249224A056182803C41C5DB38
:100B30007370043001A07370043001A0304041E2B2
:100B40001C40D5CB1C5C7D5785071CDC3C4463876F
:100B5000E7083C44854485073CC475BFBD32185C3A
:100B60005C5CAA89636DF702304079DA4844D2852B
:100B7000EF30604B3C4058441440B307F0403E9780
:100B800058C46375D7005840BA975CC48947E39B43
:100B9000F4FA1C5CC5DB1C5CFD171CDC65B730403F
:100BA00045D24844D285EF3000483C405844144078
:100BB000B307F0403E9758C4E367D7FCD9BFDDF4D4
:100BC0000844D285EF3020461C4434405840B69744
:100BD0001CC4E3E9E7F61C401CC4ADB75C50854477
:100BE0009DDB13054402EF10107F15D5E30509F2D4
:100BF000232099000DB74840EF20C02C2322040089
:100C000091B721CD3C4181C77370043001A01C41D4
:100C1000A1CB011122CC26CA2A844AC84EC606CED0
:100C20002E896530185C5C5CAA898144637DF7007D
:100C30001C5C7D5785071CDC3C446388E7023C4410
:100C4000854485073CC44E85B538F240624426850C
:100C50004249D244B249056182807370043001A0D8
:100C60005C41C5DB7370043001A05C5099E385449E
:100C7000D9BF13054402EF10107675D9E30909FEB8
:100C800085472320F900E5B7397106DE22DC26DA34
:100C90004AD84ED652D456D232C66302051C638A55
:100CA000051AB68AAE892A84EF20A01511E5B2474D
:100CB00081C77370043001A0EF2060291C5C63922F
:100CC0000714B247638E070A2808EF20E003FD549B
:100CD00013094402130A0401EF20A029EF10600C4D
:100CE000EF20E0267C4063949700232204043C44D8
:100CF0006394970023240404EF20A0276C002808A5
:100D0000EF20A00263130518EF2060241C5CADCF18
:100D1000EF202026EF20A0233C44634FF00039A8A9
:100D20004A85EF10506B19C1EF20200B3C44FD1792
:100D30003CC43C446354F0005C50FDF324C4EF20F9
:100D40004023EF20C0207C40634FF00039A852853B
:100D5000EF10706819C1EF2040087C40FD177CC07F
:100D60007C406354F0001C48FDF364C0EF20602019
:100D7000EF102028EF20A01D1C5CC1E7B247A9FF9F
:100D8000EF20201F014555A0EF20A01E1C40DDC70D
:100D9000B2454A85EF10F045EF20601B3C44634F9D
:100DA000F00039A84A85EF10106319C1EF20E00266
:100DB0003C44FD173CC43C446354F0005C50FDF3DC
:100DC00024C4EF20001BEF2080187C40634FF0000C
:100DD00039A85285EF10306019C1EF2000007C4027
:100DE000FD177CC07C406354F0001C48FDF364C0D8
:100DF000EF202018EF10E01F31C9EF2040151C5CD8
:100E0000B5DFCE8522854444EFF0CFF8639C0A0419
:100E10001C5C1840FD171CDC01E7EF20001A48C0DD
:100E20001C48A1EFEF20E0140545F2506254D25463
:100E30004259B259225A925A21618280EF202011E0
:100E40004840EF10107EEF20C01299B7EFF00FDC92
:100E50006DB73C41E38707E47370043001A0737001
:100E6000043001A05C5044C4D5DF13054402EF10E8
:100E700090564DD9EFF08FD975B713050401EF10D7
:100E800090558547E310F5FAF5B72285EFF06FF23C
:100E9000EF102016014551BF1DC9411122C44AC09F
:100EA00006C626C244412E892A84EF10D07463837B
:100EB000A40281464A8681452285F933854763002D
:100EC000F502B2402244924402494101828073708B
:100ED000043001A05C44054585075CC4DDB75C4473
:100EE00085075CC4F9BF15CDADC9011122CC26CA56
:100EF0004AC84EC652C42A8406CE3289AE89EFF063
:100F0000CFDC1C5C2A8A814485E35285EFF08FDBBD
:100F1000F240624426854249D244B249224A0561E0
:100F200082807370043001A0304001CE4C445C409C
:100F3000B2954CC463E4F5000C404CC44E85EF30D0
:100F4000800E1C5C7D57FD171CDC7C40638CE70029
:100F50007C40854485077CC04DBF3C41D9D7737028
:100F6000043001A01C4899E3854445B713050401EA
:100F7000EF10704675D9E30909FE85472320F90073
:100F8000E5B721C93C41A1CDA1CB011122CC26CA94
:100F90004AC852C42A8406CE4EC62E8AEFF0EFD23B
:100FA0001C5C2A89814491CB8329C400D285228587
:100FB000EFF04FDE8544232634014A85EFF08FD0D1
:100FC000F240624426854249D244B249224A056130
:100FD00082807370043001A07370043001A0EDDFD3
:100FE0007370043001A001E57370043001A0411159
:100FF00022C42A8406C6EF109075005CEF1070774B
:10100000B240228522444101828001E573700430A0
:1010100001A0411106C622C42A84EF1050731C5C43
:10102000405C1D8CEF10F0742285B24022444101D7
:10103000828019C1085D82807370043001A01DCDCB
:101040009787030093878779D843630CE502D847D5
:10105000630CE504D84B6307E504D84F6302E5044D
:10106000D853630DE502D8576308E502D85B6303E4
:10107000E502D85F630EE5006F20D0747370043012
:1010800001A001470E07BA9723A007006F209073B5
:101090001D47CDBF1947FDB71547EDB71147DDB760
:1010A0000D47CDB70947F9BF0547E9BF68458280BD
:1010B0006CC5828003450505828009C5085D13352E
:1010C000150082807370043001A019C51C5D485D55
:1010D0001D8D1335150082807370043001A0978731
:1010E00003009387A76F984305C3984705C7984B9C
:1010F00005C7984F05C7985305C7985705C7985B0C
:1011000015C7985F15C3828001470E07BA978CC335
:10111000C8C382800547D5BF0947C5BF0D47F5B78E
:101120001147E5B71547D5B71D47C5B71947F1BFF3
:10113000978703009387876AD8436308E502D847F7
:10114000630BE502D84B630AE502D84F6309E50259
:10115000D8536308E502D8576307E502D85B6308F4
:10116000E502D85F6303A702828001470E07BA97A2
:1011700023A0070082800547D5BF0947C5BF0D479B
:10118000F5B71147E5B71547D5B71D47C5B7194797
:10119000F1BF411122C426C24AC02A8406C6AE84C9
:1011A0003289EF10D05A7840FD576314F70023229C
:1011B00004043844FD576314F70023240404EF109B
:1011C000505B1C5C99E74A86A68513054402EF1024
:1011D0005015EF10D0573C44635BF0025C5085CB58
:1011E0009304440209A83C44FD173CC43C446350AA
:1011F000F0025C5089CF2685EF10F01D6DD5EF1001
:10120000D03D3C44FD173CC43C44E344F0FEFD5754
:101210003CC4EF101056EF1090537C40635BF0021B
:101220001C4885CB9304040109A87C40FD177CC0B1
:101230007C406350F0021C4889CF2685EF10B0191E
:101240006DD5EF1090397C40FD177CC07C40E344A5
:10125000F0FEFD577CC02244B24092440249410155
:101260006F10305197F701009387872F944317F73A
:1012700001001307A72D1843C8C2636EE502411190
:1012800022C406C617F701001307472D2A84084316
:101290008C439105EFF0CFAA97F701009387472978
:1012A0009C436376F40097F7010023A38728B2409C
:1012B00022444101828017F701001307E729084300
:1012C0008C4391056FF0CFA797F7010093874729CB
:1012D000984394437C43FD177CC3FC4299E37360BD
:1012E000043082801DC179714ECE56CA06D6BE8AA0
:1012F00022D426D24AD052CC5AC85EC69147BA8967
:1013000063F8E7007370043001A07370043001A02B
:101310002A8BAE843289B68B428A63080822130571
:101320000006EF2010382A84630C05200A092328C0
:1013300045034A869305500A5285EF20D05C03C7C7
:1013400004001C587119230AE40203C704003E99E3
:101350001379C9FF79C783C71400A30AF40283C7AE
:101360001400E1C383C72400230BF40283C72400C5
:10137000CDCB83C73400A30BF40283C73400D5C39D
:1013800083C74400230CF40283C74400D9CB83C72E
:101390005400A30CF40283C75400C1C783C7640080
:1013A000230DF40283C76400ADCF83C77400A30D7F
:1013B000F40283C77400B5C783C78400230EF40208
:1013C00083C78400B9CF83C79400A30EF40283C7F8
:1013D0009400A1CB83C7A400230FF40283C7A40009
:1013E000A9C383C7B400A30FF40283C7B40095CB8D
:1013F00083C7C4002300F40483C7C4009DC383C70C
:10140000D400A300F40483C7D40081CF83C7E400D1
:101410002301F40483C7E40089C783C7F400A30150
:10142000F404130A44005285A30104042326340360
:1014300023283405232A0404EFF0AF8E130584011A
:10144000EFF02F8E9547B3873741232C040400C853
:101450001CCC40D023220404232E04045E86DA85AB
:101460004A85EFF02F8708C063840A0023A08A0012
:101470007370043017F901001309C90C83270900A0
:1014800097F401009384C40D91C798409C407C431D
:1014900085077CC317F701001307870B1C438507DB
:1014A00097F6010023A6F60A9C40CDCB83270900BE
:1014B00089EB9C40DC5763E6F90097F7010023A114
:1014C000870A97F701009387E706984397F601008C
:1014D000938686075C549442050717F60100232B78
:1014E000E60438C463F6F60017F70100232EF7046C
:1014F0005147B387E70217F5010013056518D28538
:101500003E95EFF06F828327090089C79C40FC431A
:101510006395070E83270900054499C79C40DC5753
:1015200063F43701EFE09FEE2285B25022549254CB
:101530000259F249624AD24A424BB24B456182801B
:101540005285EF2030287D54C5B713152600EF20B3
:1015500050152A8AE31505DC7D54F9B797F7010089
:1015600023A0870018438547E31DF7F417F5010012
:1015700013050511EFE0BFF917F5010013058511FB
:10158000EFE0FFF817F5010013050512EFE03FF853
:1015900017F5010013058512EFE07FF717F501003D
:1015A00013050513EFE0BFF617FB0100130B8B13B8
:1015B0005A85EFE0DFF597FA0100938AEA13568522
:1015C000EFE0FFF417F5010013054514EFE03FF4D9
:1015D00017F501001305C514EFE07FF317F50100BF
:1015E00013054515EFE0BFF297F7010023A867F751
:1015F00097F7010023A257F7E9B5984094407C4340
:10160000FD177CC3FC42E39707F07360043019B701
:10161000411122C406C626C24AC02A84737004300F
:1016200097F40100938404F29C40F9E311E497F7E6
:1016300001009387E7F28043130944004A85EFE0F5
:101640003FF31C5489C713058401EFE07FF2CA857C
:1016500017F501001305C50CEFE01FED97F701002A
:10166000938747EF984397F701009387A7EC9C4334
:10167000050797F6010023AFE6EC9840850797F63B
:10168000010023A9F6EA01CB97F70100938747ED04
:101690009843784349EF9C40B1C797F7010093877F
:1016A00027EC9843630F870873700430984039EB38
:1016B00017F70100130787EA14439442A5E27D5708
:1016C00097F6010023A6E6E6984009CF98437843B1
:1016D00011CB984394437C43FD177CC3FC4299E3B0
:1016E00073600430B2402244924402494101828036
:1016F00097F701009387C7E698439C437C4385078F
:101700007CC32DB794439843F8420507F8C217F7F6
:1017100001001307A7E414439442D5D21843584755
:101720005847584397F6010023A4E6E071BF984359
:1017300094437C43FD177CC3FC42B1FF73600430CB
:1017400099BF97F70100938767DE9C4381C7737049
:10175000043001A02244B2409244024941016FE0AA
:10176000FFCA41C517F70100130787DF14438147FC
:10177000638BA606411106C622C426C273700430CC
:1017800097F60100938606DC9C4291C710431C43E8
:101790007C4285077CC29C42AA84404981C71C4385
:1017A000FC43B9E797F70100938747DB9C43638AC3
:1017B000870497F70100938727DA9C4363838704A4
:1017C00097F70100938707F76308F40297F7010082
:1017D000938707F56300F4028547B24022449244A0
:1017E0003E85410182803E8582807370043001A075
:1017F000E13C4DBF9147D5B79C5493B7170089077B
:10180000E9BF8947D9BF7370043097F70100938708
:1018100067D3984309EF15C59C43485581CB97F78B
:1018200001009387E7D39843784315E3828017F745
:1018300001001307E7D214431843F8420507F8C222
:1018400061FD17F701001307A7D10843F1B79843CB
:1018500094437C43FD177CC3FC42E9FB7360043076
:101860008280411122C42A8406C6EFE01FC611E41B
:1018700097F701009387C7CE80434054EFE09FC4A1
:10188000B2402285224441018280914763F5B7002E
:101890007370043001A0011122CC06CE26CA4AC8BA
:1018A0004EC652C42A847370043017F9010013091C
:1018B00069C983270900D5EF79C43C486389F508D5
:1018C00017F701001307C7C963FCB7001443638C03
:1018D000860C18434457B3B4950093C4140029A050
:1018E0000443818C93B4140058546384E70A1C4C5D
:1018F0002CC863C607009547B385B7400CCC931737
:101900002700BA97584897F90100938969D78A0741
:10191000CE97631BF702130A44005285EFE05FC5C0
:1019200017F70100130747C25C5418436376F700AA
:1019300017F70100232AF7C05147B387E702D28582
:101940003385F900EFE05FBE99C0EFE03FAC83273D
:10195000090081CB97F70100938787C09C43FC4324
:101960009DEBF2406244D2444249B249224A0561A9
:10197000828097F701009387A7BE98439C437C43DE
:1019800085077CC31DF897F70100938767BD8043E7
:101990002DB74CD4A9BF6244F240D2444249B24967
:1019A000224A056115B2814481B725C1011126CAB9
:1019B00097F401009384C4BA9C4006CE22CC4AC856
:1019C0004EC6638DA7027370043017F90100130926
:1019D00069B78327090091C798409C407C438507DD
:1019E0007CC3584997F701009387C7D46302F70275
:1019F0008327090081C79C40FC43A5EBF240624469
:101A0000D2444249B249056182807370043001A01A
:101A10001C5517F70100130767CFE38BE7FCE9FBC1
:101A2000930945002A844E85EFE09FB417F7010023
:101A3000130787B15C5418436376F70017F701006A
:101A40002324F7B05147B387E70217F501001305C8
:101A500025C3CE853E95EFE03FAD9C405854DC5702
:101A6000E368F7F8EFE09F9A61B76244F240D2442E
:101A70004249B249056189B815CD011122CC26CA67
:101A80004AC82A8406CE4EC6EFE03FA4584897F7CE
:101A90000100938727CA2A8981446300F7024A8597
:101AA000EFE05FA2F240624426854249D244B24947
:101AB000056182807370043001A01C5417F5010089
:101AC0001305C5C4E38DA7FCF9FB97F701009387C5
:101AD000E7A59C43A9EB97F70100938767A89C4370
:101AE000445493094400DC574E85B3B4F400EFE04E
:101AF0003FA817F70100130727A55C54184393C4A8
:101B000014006376F70017F70100232FF7A251475F
:101B1000B387E70217F50100130585B6CE853E951C
:101B2000EFE09FA0ADBF93058401EFE0FF9F85BF6D
:101B30000111056506CE22CC26CA4AC84EC652C43B
:101B400056C2EF200036630E051CAA84130500065A
:101B5000EF2020352A84630A051E05669305500A86
:101B600004D92685EF20205A04588567F117BE94C2
:101B7000B7474C4593879744930944005CD84E85FA
:101B8000230C0402A30104042326040223280404D2
:101B9000232A0404EFE0FF9813058401EFE07F9807
:101BA0009547232C0404F19800C81CCC40D0232274
:101BB0000404232E04040146971500009385E5B123
:101BC0002685EFE03F9108C07370043017F90100DB
:101BD000130949978327090097F4010093844498D7
:101BE00091C798409C407C4385077CC317F7010050
:101BF000130707961C43850797F6010023AAF6945E
:101C00009C40C9C38327090081EB9C40DC5789E7CE
:101C100097F7010023A6879497F701009387879190
:101C20009C4397F601009386269258549442850768
:101C300017F601002320F6903CC463F6E60097F700
:101C4000010023A3E79093172700BA978A0717F597
:101C500001001305E5A23E95CE85EFE0FF8C8327BA
:101C6000090081C79C40FC43F1E78327090091C329
:101C70009C40EF10704985476304F50E5DE1737079
:101C8000043001A097F7010023AC878C18438547E7
:101C9000E314F7F817F501001305859EEFE03F8781
:101CA00017F501001305059FEFE07F8617F501008A
:101CB0001305859FEFE0BF8517F50100130505A00B
:101CC000EFE0FF8417F50100130585A0EFE03F84E6
:101CD00097FA0100938A0AA15685EFE05F8317FA0D
:101CE0000100130A6AA15285EFE07F8217F5010017
:101CF0001305C5A1EFE0BF8117F50100130545A24B
:101D0000EFE0FF8017F501001305C5A2EFE03F806B
:101D100097F7010023A4578597F7010023AE478367
:101D2000E5BDF2406244D2444249B249224A924A55
:101D300005618280984094407C43FD177CC3FC423F
:101D4000E39507F2736004300DB76244F2404249F4
:101D5000B249224A924A2685D24405616F208026E4
:101D600073700430FD5717E701002323F77C6244AA
:101D700097E7010023A8A77CF240D2444249B24928
:101D8000224A924A97E7010023A2077C05616FE08F
:101D90004FD17370043097E7010023A5077A6FE0F5
:101DA0008FDE17E70100130767781C4385071CC304
:101DB00082807370043097E701009387A778984377
:101DC00005E317E701001307677808439C4381CBBD
:101DD00097E701009387C7789843784301EF8280A3
:101DE00017E701001307C77714431843F8420507A4
:101DF000F8C2C1BF984394437C43FD177CC3FC42A7
:101E0000F9FF736004308280411106C622C4EFE0FE
:101E1000CFEB97E70100938767738043EFE08FEA8A
:101E2000B240228522444101828097E701009387D6
:101E3000277288438280797106D622D426D24AD06E
:101E40004ECE52CC56CA5AC85EC697E70100938759
:101E5000E76D9C43B1EF17E701001307276F1C43A1
:101E6000850797E6010023A3F66E832A0700638F98
:101E70000A0697E701009387A76B9C43814463F1AF
:101E8000FA0897E901009389A97F17EA0100130A6C
:101E90002A6D83270A008546D85793172700BA97DB
:101EA0008A07BE9983A7090063FFF600854421A82D
:101EB00097E701009387C7689C438144850717E72C
:101EC0000100232FF76697E70100938727679C435C
:101ED00091C38544B2502254268502599254F24946
:101EE000624AD24A424BB24B4561828017E40100FC
:101EF0001304C4661C409C43DDC37370043001A00E
:101F000017E401001304846597E901009389497778
:101F100017EA0100130ACA6417EB0100130BCB6226
:101F20001C409C43B5C31C40DC4703A9C700832762
:101F30004900930B49005E8563EEFA04EFE04FE33E
:101F4000832789021305890199C3EFE06FE2832794
:101F5000C90203270B00DE85139527003E950A056D
:101F60004E956376F70017E70100232FF75CEFE04B
:101F7000AFDB83270A000327C902DC57E362F7FAC5
:101F80001C4085449C43C5F3FD5717E701002321FE
:101F9000F75A01B717E70100232CF758DDBD17E703
:101FA00001001307675B1C40184397E6010023A755
:101FB000E65A17E701002321F75A97E701009387B4
:101FC000A7579C43850717E701002327F7561C40B6
:101FD0009C4399E7FD5717E70100232BF75451BDA8
:101FE0001C40DC47DC47DC4317E701002322F754A1
:101FF00049B597E7010093876753984301E77370EA
:10200000043001A0011106CE22CC26CA4AC84EC611
:1020100052C456C25AC07370043097E401009384CE
:102020006452984061EB98437D1797E6010023AF17
:10203000E64E9C43D9EB97E70100938767519C4399
:10204000C9C797EA0100938AAA6317EA0100130A35
:10205000AA4F17E901001309A950854919A833852A
:10206000EA00EFE06FCC832709005854DC5763790E
:10207000F70483A7CA08C1CF83A78A09C0471305FD
:102080008401EFE0EFCE130B44005A85EFE04FCE12
:102090005C5483260A00DA85139527003E950A05CD
:1020A0002A875695E3FDF6FA17E70100232EF74835
:1020B000EFE08FC7832709005854DC57E36BF7FA2A
:1020C00097E7010023AC37476DB701449C4081CBB3
:1020D00097E701009387C7489C43FC4395E7228517
:1020E000F2406244D2444249B249224A924A024BE7
:1020F0000561828017E701001307874614431843E0
:10210000F8420507F8C205B7EFF00F9CC9BF17E406
:1021100001001304E4421C4095C31C40054999CFBB
:10212000193B09C597E7010023AA27411C40FD1769
:1021300017E701002326F7401C40FDF397E7010055
:102140009387C73F98438547E311F7F8EFE00FAC5B
:102150000544ADBF11CD81E57370043001A017E7D0
:1021600001001307A73C1C4399C77370043001A0FA
:102170007370043001A0411122C406C614431841F3
:10218000850617E601002323D63A97E601009386D9
:10219000E63B94423304B70000C163F7E602637F75
:1021A000E40063FD860097E701009387673B88435F
:1021B0001105EFE0EFBB2285EFF0CF8A1D3D01C98D
:1021C000B240224441018280E36FE4FCD9BF224443
:1021D000B24041016FE08FA311C917E70100130757
:1021E000E7341C4391C77370043001A06FE00FA265
:1021F000411106C622C41843AA87050797E60100C5
:1022000023A6E63297E601009386863517E701009C
:102210001307C733184388423304F7001105EFE072
:102220002FB52285EFF00F84E93311E52244B24047
:1022300041016FE0AF9DB2402244410182804111D3
:1022400022C406C697E701009387472E9C430144AA
:10225000850717E70100232BF72C97E701009387E9
:10226000272F9C4363E3F50C17EE0100130ECE46B7
:1022700097E201009382024001440147854F130316
:10228000500A21A0311E6387C20D83278EFFBA85B5
:10229000F5DB8327CEFFDC43232EFEFE6382C71BC4
:1022A00003AFC700DC432A97814E232EFEFE6385D1
:1022B000C70783A8C70093874803232017015CC37F
:1022C00083A788042326F7011CC783A7C8021CCB59
:1022D00083A70805232C07005CCB03A808038347CA
:1022E0000800639A6704C287850783C60700B38521
:1022F0000741E38B66FE8981C205C181231EB700B9
:10230000850E1307070263001F058327CEFFDC43FA
:10231000232EFEFEE39FC7F983274E00232EFEFEE9
:1023200049BF1A9419C223200600E1312285B24028
:102330002244410182808145231EB700850E130788
:102340000702E3141FFD769413175400311EBA855B
:10235000E39DC2F397E701009387472003AE070090
:1023600083270E00FDE397E701009387E71E03AE86
:10237000070083270E006398071617EE0100130E5F
:102380002E3083270E0A639D071E83274E0BD9DB51
:1023900083278E0B97EE0100938E4E3ADC4317E7AE
:1023A0000100232BF7386381D73383AFC700DC43A9
:1023B0003307B500014397E6010023AFF6360D4F12
:1023C00089429308500A6386D707C8479307450395
:1023D00008C35CC33C452326E7011CC75C551CCBE6
:1023E0001C5599C3232657003C49232C07005CCB7E
:1023F00003280503834708006395172BC2878507C9
:1024000083C60700B3850741E38B16FF8981C205A8
:10241000C181231EB700050313070702E383AFF052
:1024200083278E0BDC4397E6010023A7F630E39E5B
:10243000D7F983270E0C97E6010023AFF62E71B76C
:1024400083274E00232EFEFEA1BD83274E00130FCF
:102450008E00D4432322DE00638CE625B307E5001B
:10246000D84283A2C600814E2322EE00894F130377
:10247000500A6305EF068328C7001387480323A08B
:102480001701D8C303A7880423A6F70198C703A799
:10249000C80298CB03A7080523AC0700D8CB03A834
:1024A0000803034708006318671C42870507834633
:1024B0000700B3050741E38B66FE8981C205C18130
:1024C000239EB700850E93870702638E121B832617
:1024D0004E00D8422322EE00E31FEFF80327CE0080
:1024E0002322EE0049BF83274E00130F8E00DC43EA
:1024F0002322FE006389E71B83A2C700DC43AA9561
:10250000814E2322FE00894F1303500A6305FF0604
:1025100083A8C7009387480323A01501DCC183A7C4
:10252000880423A6F5019CC583A7C8029CC983A77C
:10253000080523AC0500DCC903A80803834708008D
:1025400063976710C287850783C6070033870741F3
:10255000E38B66FE098342074183239EE500850ED7
:1025600093850502638D120F83274E00DC432322DF
:10257000FE00E31FFFF88327CE002322FE0049BFA1
:1025800083274E0A17EF0100130F0F1ADC4317E7DA
:1025900001002329F7186382E71383A2C700DC43F5
:1025A000AA95814E17E70100232EF716914F1303CA
:1025B000500A6387E70783A8C7009387480323A0CF
:1025C0001501DCC183A7880423A6F5019CC583A758
:1025D000C8029CC983A7080523AC0500DCC903A871
:1025E00008038347080063946704C287850783C68E
:1025F000070033870741E38B66FE09834207418367
:10260000239EE500850E93850502638A12038327C6
:102610004E0ADC4317E701002326F710E39DE7F994
:102620008327CE0A17E70100232EF70E69B701476B
:10263000239EE500850E93850502E39A12FD83270C
:102640004E0B769493155400E38E07CC91B301475B
:10265000239EE500850E93850502E39712F117EEA0
:102660000100130EEE0183270E0A76949315540091
:10267000E38D07D031B78145239EB700850E938740
:102680000702E39612E597E701009387E7EC03AEB4
:10269000070076949315540083270E00E38F07CC30
:1026A00099B58145BDB38327CE002322FE00A9B58D
:1026B0008326CE002322DE0055B38327CE0A17E7F8
:1026C00001002321F706D1BD83270E0C17E7010077
:1026D0002324F706D9B9797126D24AD04ECE52CCEE
:1026E00056CA5AC85EC606D622D497E90100938915
:1026F000E9E317E901001309A9F817EA0100130A31
:102700006AE497EA0100938AAAE597EB0100938BAC
:102710002BE497E401009384E4E3054B21A883A70D
:1027200009000324090A850717E701002320F7E0C1
:10273000C93011E89C40E5F783270900E37CFBFEE4
:10274000EFD0DFCCC5BF7370043083270A00B9E334
:102750008327C90AC04713054400EFD07FE183A750
:102760000B00FD1717E701002324F7DE9C40FD173F
:1027700017E701002320F7DE83270A0089C783A714
:102780000A00FC4385E30858EF10D0032285EF10C0
:1027900070034DB703A70A0083A70A007C4385078F
:1027A0007CC37DB703A70A0083A60A007C43FD17FC
:1027B0007CC3FC42E9FB73600430F1B797E701008A
:1027C0009387C7D69C43DDE3411106C697E7010016
:1027D00023A607D617E70100130787D81C43B7A61F
:1027E000A5A59386565A9C5B8C43639BD500D0432A
:1027F0006318B60094476395C600DC476388D7002A
:1028000008430C4393854503EF20700097E60100D1
:10281000938686D3904217E70100130767E611A855
:102820009C42B9CB9C42FD1717E60100232EF6D03F
:10283000904293172600B2978A07BA979C43EDD32C
:10284000904293172600B2978A07B305F700D44148
:10285000A107BA97D442D4C16383F602DC46B240E2
:1028600017E70100232EF7CE41018280854717E745
:1028700001002325F7CC82807370043001A0D1477A
:102880003306F602D442329754C3C9BF01114AC875
:1028900006CE22CC26CA4EC62A897370043097E42D
:1028A0000100938424CA9C4017E40100130444CB24
:1028B000D9E76314090003290400930949004E85F0
:1028C000EFD01FCB8327890289C713058901EFD079
:1028D0003FCACE8517E501001305C5E5EFD0DFC47B
:1028E0009C4081C71C40FC43ADE31C40638B270721
:1028F0009C409DCF737004309C40C1EB97E7010072
:102900009387C7C59843184325EBFD5717E7010088
:102910002320F7C29C4089CF1C40FC4391CB184038
:1029200014407C43FD177CC3FC4299E37360043080
:10293000F2406244D2444249B24905618280184063
:102940001C407C4385077CC3ADB7184014407C43D2
:10295000FD177CC3FC42D1FB736004301C40E3993B
:1029600027F99C40A1C397E70100938727BC9C43AC
:10297000ADCB7370043001A09C43DC47DC47DC43E3
:1029800017E701002326F7BA71B718401C407C43B3
:1029900085077CC397E70100938747BC984318439A
:1029A0002DD7D9BF97E70100938787BA17E70100B2
:1029B000130707CD9C430327470B631DF700F24025
:1029C000624497E7010023AD07B8D2444249B249B7
:1029D000056182806244F240D2444249B2490561B5
:1029E000F1BB6244F240D2444249B24905616FD022
:1029F000FFA13DC9411126C297E40100938444B66A
:102A00004AC02E898C4006C622C4E105EFD05FB3D0
:102A100088401105EFD0DFB5FD57630AF90497E749
:102A200001009387A7B2804398409C434A9440C3D7
:102A3000636CF40497E70100938747B288438C40A6
:102A40009105EFD0FFAF97E70100938767AE9C43F6
:102A50006376F40097E7010023AC87ACB2402244D0
:102A600092440249410182807370043001A08C407D
:102A70002244B2409244024917E50100130585CB78
:102A8000910541016FD05FAA97E701009387C7AC1A
:102A9000884322448C40B24092440249910541014E
:102AA0006FD01FAA11C997E70100938727A89C43FD
:102AB00099E77370043001A07370043001A04111D4
:102AC00026C297E401009384A4A99840AE878C4065
:102AD000B7060080D58F06C622C41CCFE10532841C
:102AE000EFD09FA488401105EFD09FA8FD57630E3B
:102AF000F40097E70100938767A58843B2409244AA
:102B00002295224441016FE0EFF58C402244B2400F
:102B1000924417E501001305E5C1910541016FD00D
:102B2000BFA025CD411126C297E40100938444A3A0
:102B30004AC02E898C4006C622C4E1053284EFD0FB
:102B4000BF9E88401105EFD0BFA28547630AF404F9
:102B500097E701009387879F804398409C434A945E
:102B600040C3636CF40497E701009387279F884371
:102B70008C409105EFD0DF9C97E701009387479B3E
:102B80009C436376F40097E7010023A3879AB24041
:102B9000224492440249410182807370043001A0B2
:102BA0008C402244B2409244024917E501001305CB
:102BB00065B8910541016FD03F9797E70100938772
:102BC000A799884322448C40B2409244024991051F
:102BD00041016FD0FF96411106C622C426C25C4552
:102BE000C04735CC930484012685EFD07F9897E7C2
:102BF00001009387A7939C43B5E79304440026857F
:102C0000EFD01F9797E701009387079458549C4390
:102C100063F6E70097E7010023A8E79293172700E0
:102C2000BA978A0717E50100130585A5A6853E9585
:102C3000EFD09F8F97E70100938787929C4358546A
:102C40000145DC5763F8E700854717E701002327B4
:102C5000F78E0545B2402244924441018280737050
:102C6000043001A0A68517E50100130525AAEFD0C1
:102C7000BF8BC9B797E701009387478B9C4381E7D8
:102C80007370043001A0411106C622C426C2B707E2
:102C900000804045CD8F1CC12DC4EFD07F8D9304A3
:102CA00044002685EFD0DF8C97E701009387C78922
:102CB00058549C4363F6E70097E7010023A6E78892
:102CC00093172700BA978A0717E501001305459B5C
:102CD0003E95A685EFD05F8597E7010093874788EB
:102CE0009C4358540145DC5763F8E700854717E7D4
:102CF00001002325F7840545B24022449244410156
:102D000082807370043001A011CD97E70100938792
:102D1000A782984397E70100938747839C4318C194
:102D20005CC182807370043001A055C1D1CD4111C6
:102D300006C622C42A877370043097E8010093887E
:102D4000688083A7080091CB97E7010093874781AC
:102D500094439C43FC428507FCC217D30100130334
:102D6000E37E9C4103260300FD560144638FD70296
:102D700017DE0100130E4E7C03250E00032807000A
:102D800054436305A80005446371D6023308D64056
:102D90000544637CF80003250E00918F0326030091
:102DA000B6979CC108C350C3014483A7080081CBD8
:102DB00097D701009387C77A9C43FC4381EF228514
:102DC000B2402244410182807370043001A07370CC
:102DD000043001A0EFE04FCFDDB7854717D70100E2
:102DE000232EF774828019C1684582800145828054
:102DF00011C16CC5828097D701009387677688439D
:102E0000828097D701009387E7739C43054589CB60
:102E100097D70100938787718843133515000605FE
:102E2000828031CD011126CA97D401009384447366
:102E30009C4006CE22CC4AC84EC65855DC57637912
:102E4000F7021C4D63C707009C40D4579547958FE8
:102E50001CCD93172700BA97584917E901001309A9
:102E600029828A07CA97630DF7009C40DC575CD51E
:102E7000F2406244D2444249B24905618280828074
:102E8000930945002A844E85EFD08FEE9C4017D7DA
:102E900001001307676B1843DC575CD46376F700B7
:102EA00017D701002322F76A139527003E95624445
:102EB0000A05F240D244CE854A95B249424905619D
:102EC0006FD08FE619CD411106C622C426C297D70E
:102ED00001009387E76880436307A40073700430A0
:102EE00001A0014582807C4881E77370043001A015
:102EF00054543848FD177CC86383E60099C70145E0
:102F0000B2402244924441018280930444002685C9
:102F1000EFD00FE63C4817D701001307E7621443D0
:102F200015471D8F5CD418CC63F6F60017D7010047
:102F3000232CF7605147B387E70217D5010013052B
:102F40002574A6853E95EFD02FDE054555BF7370DD
:102F5000043097D701009387E75E9C4391CB97D7C6
:102F600001009387E75F98439C437C4385077CC3BC
:102F7000828097D701009387E75C9C438DC397D7E6
:102F800001009387E75D9843784311CB98439443BE
:102F90007C43FD177CC3FC4299E37360043082805C
:102FA00097D701009387C75B904394439843954715
:102FB000D456084E958F1CCF828097D701009387F7
:102FC000275A984309C79443F84A0507F8CA884323
:102FD000828079714AD006D622D426D24ECE2A8952
:102FE0007370043097D401009384C4559C4017D467
:102FF00001001304E456BDE31C40BC4F89E71C40AC
:103000000547F8CFD1E19C4081C71C40FC43F1EB60
:10301000737004309C408DEF1C40A84F11C56304B1
:1030200009021C4023AC07041C4023AE07049C404B
:1030300081C71C40FC438DEBB2502254925402597C
:10304000F2494561828018403C4FFD173CCFE9BFF3
:1030500018401C407C4385077CC37DBF18401C4042
:103060007C4385077CC349BF184014407C43FD174F
:103070007CC3FC42F1F373600430B250225492548A
:103080000259F2494561828008402EC61105EFD0F1
:103090002FCEB245FD576380F50697D70100938781
:1030A000E74A83A9070018409C43AE9923223701C1
:1030B00063ECF90497D701009387474A88430C4093
:1030C0009105EFD0EFC797D70100938767469C43E0
:1030D00063F6F90097D7010023AC3745EFD00FB363
:1030E0001DB7184014407C43FD177CC3FC428DF390
:1030F0007360043031BF0C4017D5010013058563A0
:103100009105EFD06FC2D9BF97D701009387C7440D
:1031100088430C409105EFD0AFC2C9B779714AD04E
:103120004ECE06D622D426D252CC2E89B2897370C6
:10313000043097D401009384E4409C4017D40100EC
:1031400013040442F9EF18408947784F630CF700E5
:103150001C401345F5FFB84F798DA8CF1C4005479B
:10316000F8CFADE69C4081C71C40FC43F5E373708B
:1031700004309C40B1E7638609001C40BC4F23A08B
:10318000F900184085470145784F630BF7001C4054
:103190001349F9FF0545B84F3379E90023AC2705FA
:1031A0001C4023AE07049C4081C71C40FC43C1E384
:1031B000B250225492540259F249624A45618280C7
:1031C00018401C407C4385077CC375B7084036C651
:1031D0001105EFD0EFB9B246FD576385F60897D7D2
:1031E00001009387A73603AA070018409C43369A2C
:1031F000232247016363FA0897D7010093870736B4
:1032000088430C409105EFD0AFB397D70100938767
:1032100027329C436370FA0697D7010023AA4731EF
:1032200091A818401C407C4385077CC329BF1840E7
:1032300014407C43FD177CC3FC42BDFB736004302B
:10324000B250225492540259F249624A4561828036
:10325000184014407C43FD177CC3FC4289FB73601B
:10326000043031B70C4017D501001305A54C91056A
:10327000EFD08FABEFD08F99F5B597D7010093873B
:10328000A72D88430C409105EFD08FABE5B751C116
:10329000411106C622C426C24AC07370043097D4B6
:1032A00001009384242A9C40B9EB99C23C4D9CC2F6
:1032B000B2878946704D74CD2E872A846386D706DF
:1032C00063FCF6048D456387B70091456395B700AD
:1032D0006300D60C38CC8547630FF60405449C4048
:1032E00081CB97D701009387A7279C43FC43A9E391
:1032F0002285B2402244924402494101828097D7FC
:1033000001009387E72598439C437C4385077CC352
:1033100069BF7370043001A08546E39ED7FA3C4D27
:1033200033E7B70038CD45BF3C4D85073CCD65B789
:10333000EFD09FF975BF130944004A85EFD04FA322
:1033400017D70100130747205C5418436376F70032
:1033500017D70100232AF71E5147B387E70217D575
:1033600001001305E531CA853E95EFD0EF9B1C5453
:1033700081C77370043001A097D701009387471E5F
:103380009C435854DC57E3FBE7F4EFD02F88B9B7E0
:103390000144B1B739CD011122CC26CA4AC84EC664
:1033A00052C456C206CEBA89368AB2842E892A847D
:1033B000EFD0AF91AA8A63050A003C4C2320FA00A3
:1033C000784C89477CCC6389F40263F4970C8D4672
:1033D0006387D40091466396D400630AF70A232CCE
:1033E00024058547631EF7061C5499CB737004307F
:1033F00001A07370043001A03C4C85073CCCD5B7CC
:1034000097D70100938787129C43ADEB9304440048
:103410002685EFD0EF9517D701001307E7125C540C
:1034200018436376F70017D70100232FF710514791
:10343000B387E70217D5010013058524A6853E95BD
:10344000EFD08F8E97D70100938787119C435854F4
:10345000DC5763F7E70063850900854723A0F9007F
:1034600005445685EFD00F862285F2406244D2444F
:103470004249B249224A924A0561828093058401F9
:1034800017D5010013058528EFD00F8A65BF0144C9
:10349000C9BF8547E397F4F43C4C33E92701232C5B
:1034A000240581B74DC1011122CC26CA2A844AC8FD
:1034B00006CE4EC6AE84EFD04F818947744C7CCC8B
:1034C0003C4C05472A8985073CCC6395E6061C548D
:1034D00081C77370043001A097D701009387070557
:1034E0009C43ADE7930944004E85EFD06F8817D712
:1034F0000100130767055C5418436376F70017D77C
:1035000001002323F7045147B387E70217D50100D1
:1035100013050517CE853E95EFD00F8197D7010093
:10352000938707049C435854DC5763F5E70099C020
:1035300085479CC06244F240D244B2494A85424920
:1035400005616FC03FF87370043001A093058401DA
:1035500017D501001305851BEFC01FFDC1B7AA8752
:1035600029C57370043017D701001307A7FD144352
:103570009DE2F04F894601456315D60023AE07044E
:1035800005451C4381CB97D70100938767FD98437E
:10359000784315E3828097D60100938666FC9042BB
:1035A00094427442850674C2E9B797D701009387A5
:1035B00027FB9C437DB7984394437C43FD177CC312
:1035C000FC42E9FB7360043082805D71A6C2CAC010
:1035D00052DC56DA5AD85ED686C6A2C44EDE62D413
:1035E00066D26AD017D90100130989F817DB0100E8
:1035F000130B4BF797D40100938404F797DA01007B
:10360000938ACAF6054AA54B8327090098436301AC
:103610000712DC4783A90700EFE0AFF8EFE06FF98E
:1036200083270B002A8C6362F50A97D7010023AB2E
:10363000A7F201466370351B8840B3858941EFD0FE
:103640005FB5EFE01F9B630105128840814601468C
:103650002C00EFD06FE34DD9A247E3C807FEC24963
:1036600083A7490189C713854900EFC07FF0EFE0C8
:103670004FF483270B002A8C636DF508A24717D7F8
:103680000100232187EFE3E2FBFCB317FA0013F7F5
:103690000721631A071613F7770C6318071E93F7B1
:1036A0000702C5D74E85EF00F01145B7DC47C0478C
:1036B00083AC0700930944004E85EFC07FEB5C505C
:1036C000228582975C4C6384470B832709009843CB
:1036D00071FF03A70A0097D6010023A586E997D6B4
:1036E000010023A5F6E897D7010023A3E7E8EFE060
:1036F0005F90A1BFDC47C04703AD0700930C4400B7
:103700006685EFC0FFE65C50228582975C4C63863D
:10371000470983270900984371FF03A70A0097D63A
:10372000010023A5F6E497D7010023A3E7E4B9B786
:10373000EFE02FE7EFE0EFE783270B002A8CE3664B
:10374000F5F883A70A00884081499043B3858941F1
:1037500017D70100232887E113361600EFD07FA387
:10376000EFE03F89E31305EEEFC05FCAF9BD1C4CE3
:10377000CE85E69763E9FC049C4089CF02CA66CCFB
:1037800022CEEFF00FE88840814601464C08EFC09A
:103790009FFF05FD7370043001A01C4CE685EA977D
:1037A000636CFD049C4089CF02CA6ACC22CEEFF044
:1037B0004FE58840814601464C08EFC0DFFC31F9F7
:1037C0007370043001A0032509005CC000C8EFC07D
:1037D0003FD7E5BDEFE0FF8183270900DC47C04705
:1037E000930C44006685EFC0BFD85C4C638F4703E1
:1037F0005C502285829791BD032509005CC000C8FA
:10380000EFC01FD439B7B24723ACF900A5CFE29778
:1038100023A2F90023A8390193854900636FFC04B2
:1038200003A50A00EFC0DFD10DB51C4C00C83387DB
:10383000F90058C0636DEC02330C3C416363FC0239
:103840009C4089CF02CA4ECC22CEEFF08FDB88405D
:10385000814601464C08EFC01FF359F973700430DC
:1038600001A003A50A00E685EFC09FCD51B703254F
:103870000900E685EFC0DFCCA5BF03250900EFC036
:103880003FCCE1B37370043001A0B24783A6890135
:1038900023A839013387D70023A2E9006364EC042D
:1038A000B307FC4063EBD70483A749024E85829798
:1038B00083A7C901E39B47D983A68901B2479840F2
:1038C000B69711CF02CA3ECC4ECEEFF08FD38840D0
:1038D000814601464C08EFC01FEBE31805D6737014
:1038E000043001A06374FC00E370F7FC03250900B9
:1038F00093854900EFC0DFC489BB03A50A00938507
:103900004900EFC0FFC391B3411122C406C626C2CD
:103910004AC017D40100130424C5EFF04FE31C4044
:1039200095CBEFF00FE51C409DC3814801488147CE
:10393000094781461306004097D50100938505A8E5
:10394000170500001305A5C8EFD0DF9939E973709A
:10395000043001A017D90100130909DF4A85EFC01F
:103960001FBB97D40100938464DF2685EFC03FBA64
:103970000146B145114597D7010023AB27BF97D723
:10398000010023A597BEEFC07FD317D70100232DD9
:10399000A7BC11CD97D501009385C5A1EFD02FF419
:1039A00049B7B24022449244024941018280737077
:1039B000043001A0A5C9797156CAAA8A1305C002AC
:1039C00022D426D24AD04ECE52CC06D65AC85EC693
:1039D0003A89B689328AAE84E9212A8405C9EFF092
:1039E0000FD797D70100938727B89C439DCFEFF05F
:1039F0004FD8130544002320540104CC232E440146
:103A00002320340323222403EFC0BFB12285B25008
:103A1000225492540259F249624AD24A424BB24B62
:103A2000456182807370043001A097DB0100938BA5
:103A3000ABD15E85EFC0BFAD17DB0100130B0BD21E
:103A40005A85EFC0DFAC0146B145114597D701005B
:103A500023A077B397D7010023AA67B1EFC01FC691
:103A600017D701002322A7B001C997D5010093857C
:103A70006594EFD0CFE6A5BF7370043001A039C5BF
:103A8000011122CC06CE26CA17D401001304C4ADFE
:103A9000832804002A88014563850802BA842EC25F
:103AA000368732C442C6954663C5B602EFF06FB59D
:103AB0008947630BF5020840814601464C00EFC080
:103AC0009FCCF2406244D24405618280737004301E
:103AD00001A04C0081463A864685EFD00F80F24027
:103AE0006244D244056182800840814626864C00AB
:103AF000EFC07FC9F9B719C10841828073700430E3
:103B000001A001E57370043001A0411106C622C472
:103B10002A84EFF0CFC348483334A000EFF06FC5DC
:103B20002285B24022444101828001E57370043055
:103B300001A0411122C42A8406C6EFF04FC10050F3
:103B4000EFF02FC3B240228522444101828001E57B
:103B50007370043001A0411122C426C22E84AA84AD
:103B600006C6EFF0CFBE80D02244B240924441015D
:103B70006FF02FC04111714522C406C61D262A844C
:103B800011C5232005001105EFC07F982285B240A2
:103B900022444101828001CDB70700FFED8F81C72C
:103BA0007370043001A099E57370043001A0737044
:103BB000043001A0011122CC4AC84EC652C456C2DC
:103BC00006CE26CABA893689B28A2E842A8AEFF0AE
:103BD0004FA311E5638509007370043001A0EFE085
:103BE0004F9C83240A00B37794006316090295C79B
:103BF00063870A009347F4FFE58F2320FA00EFE084
:103C00004FBFF240624426854249D244B249224A1B
:103C1000924A05618280E30DF4FCE38209FEB3352C
:103C20005001E20563050900B7070004DD8D4E86EB
:103C3000C18D13054A00EFE0FFE6EFE08FBB19E10D
:103C4000EFC0CFFCEFF0CFB593176500AA8963D81A
:103C50000700B7040001FD14B3F499005DB7EFF05D
:103C60000FAF83290A00B3773401631E090089CBA3
:103C700063880A009347F4FFB3F737012320FA0063
:103C8000EFF02FAFF9B7E31DF4FEDDB701C9B707B9
:103C900000FFED8F99C77370043001A0737004307A
:103CA00001A0411122C42A8406C626C24AC02E8918
:103CB000EFF0EFA904409345F9FFB3F795001CC05E
:103CC000EFF02FABB24022442685024992444101D5
:103CD0008280411122C42A8406C6EFC00FFF004033
:103CE000EFC04FFEB240228522444101828009C9C3
:103CF000370700FFB3F7E50099C77370043001A0E0
:103D00007370043001A06F20100EB70700FFF18F11
:103D100081C77370043001A001E67370043001A004
:103D2000011122CC4AC84EC652C406CE26CA3689D4
:103D3000AE892A8A3284EFF0CF8C21E16305090035
:103D40007370043001A0EFE0CF8583240A00CE8594
:103D50005285B3E49900613FB37794006307F4069A
:103D600083240A00EFE0EFA8F2406244268542492E
:103D7000D244B249224A05618280EFE08F828324D7
:103D80000A00CE855285B3E434019537B3F7840039
:103D9000638D8702E30609FCB70500054A86C18DDD
:103DA00013054A00EFE01FD0EFE0AFA419E1EFC028
:103DB000EFE5EFF0EF9E93176500AA8463DF07003D
:103DC000B7070001FD17FD8C45B783270A00134490
:103DD000F4FFE18F2320FA0071B7EFF04F978324AF
:103DE0000A00B3779400639787009347F4FFE58F49
:103DF0002320FA00EFF0EF97E1B7411122C406C685
:103E00002A8426C2EFD0FFF95C4085C3084893049A
:103E1000C4006316950015A0084863009502B70515
:103E20000002EFE03FE55C40E5FB2285612A224489
:103E3000B240924441016FE0CF9B7370043001A007
:103E400009C9370700FFB3F7E50099C7737004305D
:103E500001A07370043001A06F20E07801C9B7079A
:103E600000FFED8F99C77370043001A073700430A8
:103E700001A0411122C426C206C62A84AE84EFF0F6
:103E80000F8D184093C7F4FFF98F1CC02244B24035
:103E9000924441016FF0EF8D19C1084D82800145B8
:103EA0008280411122C406C62A84EFD09FEF97C7B3
:103EB00001009387276C9C43A1EBE56717D70100AE
:103EC0001307478BF11797C6010023ABE66A17C7A4
:103ED00001002325F76A17D70100232FF78897C71A
:103EE00001009387676917D701002325F788854765
:103EF00017C701002328076817C70100232E07668C
:103F000017C701002328F76619E8EFE08F8EEF103E
:103F1000800F01442285B240224441018280130572
:103F2000840093773500C1EFE5671307F5FFE917C4
:103F3000E3EDE7FC97C60100938686649C4229A0C6
:103F4000984311C7BE86BA87D843E36BA7FE17C74D
:103F5000010013076762E38AE7FA98434146138436
:103F6000870098C2D843B306A7406378D602338847
:103F7000A7002322D800C8C38325480097C60100A4
:103F80009386066011A0BA8698425043E36DB6FE50
:103F90002320E80023A00601D84397C70100938798
:103FA00027659C43998F17C701002323F764EFE02F
:103FB0004F8431DC2285B2402244410182807199D4
:103FC00011059DB729C9411122C406C62A84EFD024
:103FD0005FDD930584FF0326C4FF17C701001307A5
:103FE000275A11A03E871C43D443E3EDC6FE232C81
:103FF000F4FE0CC397C701009387875F984383271C
:10400000C4FF2244B240BA9717C701002322F75ECB
:1040100041016FD01FFE828097C701009387475DE3
:104020008843828082803367B5000D8BAA871DE7A5
:104030009308D6FFAA982A87AE866371150303A852
:10404000060011079106232E07FFE36A17FF934727
:10405000F5FFC697F19B9107BE95AA972A9663F341
:10406000C70A9386450013884700B3B6D70033B814
:10407000050133E7F50093C61600134818000D8BB1
:10408000B3E6060113371700758F330EF64093869B
:10409000170029CF1337AE0031EB13532E002E88B3
:1040A000BE860147832808000507110823A01601D2
:1040B0009106E36967FE1377CEFFBA95BA9763025C
:1040C000EE0483C60500138717002380D700637AA8
:1040D000C70283C6150013872700A380D700637229
:1040E000C70203C725002381E7008280B307F6409B
:1040F000AE97850503C7F5FF8506238FE6FEE39A95
:10410000F5FE82808280B367C5008D8BB308C50041
:10411000E9C36371150FB307A0408D8B1387370078
:10412000954693F5F50F130815003383A8407D16C7
:104130006373D70015476363E60CD5CF2300B50042
:104140000547638DE700A300B5000D471308250060
:104150006396E700130835002301B5001396850028
:104160004D8E13970501518F3303F34093968501CC
:10417000D98E13562300AA97014794C305079107C8
:10418000E36DC7FE1377C3FFB307E8006307E306D9
:104190002380B70013871700637C1703A380B70041
:1041A00013872700637617032381B700138737002F
:1041B00063701703A381B70013874700637A170161
:1041C0002382B7001387570063741701A382B700D7
:1041D000828093F5F50F13978500D98D139705010C
:1041E0004D8FE37715FFAA87910723AEE7FEE3ED36
:1041F00017FF828082802A8895B78280AA8749BF6C
:10420000834705002A8799C7050583470500EDFF09
:10421000198D82800145828005058347F5FF85055C
:1042200003C7F5FF91C7E389E7FE3385E740828046
:104230008147E5BFAA87850503C7F5FF8507A38FDB
:10424000E7FE75FB828083460500930700026397B3
:10425000F600050583460500E38DF6FE938756FDBF
:1042600093F7D70F85C7AA87814585CE0145850776
:10427000138606FD1317250083C607003A95060529
:104280003295F5F699C13305A0408280938536FDBD
:104290008346150093B5150093071500E1FA014513
:1042A000D5B7014582809C412380A7009C418507AA
:1042B0009CC1828097C601009386062D9C421757A9
:1042C00003001307274C13861700BA972380A70013
:1042D00097C5010023AAC52AA9476308F5009307DB
:1042E00000046305F6000145828075DE370610F094
:1042F00005078347F7FF2320F6F09C42FD1797C57B
:10430000010023A3F528EDF7014582804D7123229A
:10431000911423202115232A5113232481132326AA
:10432000111423248114232E3113232C4113232809
:10433000611323267113232291132320A113232E0B
:10434000B111AA842E8932C6130C5002A54A8347A4
:10435000090063808703B9CB804011A0A1CB230063
:10436000F40080400509050480C083470900E397F5
:1043700087FF0346190093081900C686130D000233
:10438000FD597D5A0148130550059307D6FD93F753
:10439000F70F138916006363F52A17C70100130787
:1043A00067C68A07BA979C43BA9782878320C1144D
:1043B0000324811483244114032901148329C11384
:1043C000032A8113832A4113032B0113832BC11268
:1043D000032C8112832C4112032D0112832DC11154
:1043E00071618280A14C02C4854763D50715B2472D
:1043F0008040938B770093F68BFF03AB060083A975
:104400004600938786003EC6668681465A85CE85DD
:10441000EF1030682AC8814763853723930D410127
:10442000854B668681465A85CE85EF10B030814631
:1044300066862A8BAE89EF10D065A24723A0AD0017
:1044400093861B00910D63843701B68BD9BFE37E41
:104450009BFF63DD4601A2872380A70180407D1A70
:10446000930714009CC03E84E3C846FF93962B003C
:104470001C08BE9631A8938777052300F40080407E
:10448000FD1B93871B00050480C0F116E351F0EC7F
:104490009C42E3E2FAFE93870703C5B79C4093066C
:1044A000000332472380D7009C4093064700C14C4D
:1044B0001386170090C013068007A380C7008040B2
:1044C00002C4BA87050480C003AB0700814936C621
:1044D00025BFB24783AC0700938B470063840C1C55
:1044E000635F40199307D0026319FD1683C70C0060
:1044F00085C363DC09189440850C7D1A2380F6007F
:104500008040050480C083C70C00E5F7635D40016F
:104510008040930700022300F40080407D1A0504C8
:1045200080C0E31A0AFE5EC61DB502C48547A94CC9
:10453000E3CF07EBB24780409386470071B703C6CD
:104540001600CA8699B59C40930650022380D70076
:104550008040050480C0E5BBC14C02C471B5B247C0
:1045600003C61600CA8683A9070091073EC6E35E0C
:104570000AE04E8AFD5911BD03C61600130DD00284
:10458000CA8621B59347FAFFFD8703C61600337A22
:10459000FA00CA86DDBB03C61600130D0003CA86E7
:1045A000EDB383C51600930906FDCA86938705FD02
:1045B0002E86E3EEFAFA93972900BE9985068609BE
:1045C000AE9983C50600938909FD938705FD2E8664
:1045D000E3F3FAFE69BF32479C40144311073AC621
:1045E0002380D7008040050480C095B3854763D3FE
:1045F000070BB24793867700E19A938786003EC601
:1046000083A946009C4263DC090A94401306D00249
:10461000B307F0402380C6008040B336F000B309F2
:104620003041050480C03E8BB389D940A94C02C4F7
:10463000E1BB03C616000508CA8681BB9C404689BB
:1046400021B7E37D9BDD8547814B8546E3C547E187
:1046500031BD97CC0100938CECD6CE856685EF10EA
:104660004053330AAA40635C400180402300A40108
:1046700080407D1A050480C0E31A0AFE014A83C700
:104680000C00E38207EAE3C809E6FD197D57E394CD
:10469000E9E6ADBDB247938647009C4336C693D941
:1046A000F74195B7635640019307D002E313FDFA33
:1046B00097CC0100938C0CD1930780021DBD3E8BDB
:1046C000A94C02C4804089B34D71232E3113B70920
:1046D00000409387F9FF2324811423229114232C73
:1046E0004113232A51132326111423202115232893
:1046F0006113232671132324811323229113232072
:10470000A113232EB1112A8A2EC417C40100130449
:10471000A4E7975A0300938AEA0697C4010093849A
:10472000E4A33EC693055002294513080004B706CA
:1047300010F083470A006386B704C1C71840050A12
:1047400013061700569797C8010023AFC8E223004D
:10475000F7006382A706E31E06FD17570300130741
:10476000670205078347F7FF23A0F6F01C40FD17FB
:1047700017C60100232AF6E0EDF783470A00E39EFF
:10478000B7FA83461A0013051A002A87930B000212
:104790007D5B7D5C014893055005A5489387D6FD58
:1047A00093F7F70F130A170063E7F5348A07A69704
:1047B0009C43A6978287175703001307A7FC55F25F
:1047C0008DBF8320C1140324811483244114032941
:1047D00001148329C113032A8113832A4113032B54
:1047E0000113832BC112032C8112832C4112032D40
:1047F0000112832DC11171618280A14C014D854749
:1048000063DB0719A2479D07E19B83AD070003AB5C
:104810004700138787003AC4668681466E85DA852D
:10482000EF1030272AC863066D3513094101854909
:10483000668681466E85DA85EF10C06F6686814692
:10484000AA8D2E8BEF10F0242320A90085091109D1
:10485000E3106DFFE3FE9DFD13060004B70610F0A4
:1048600063D189031C4013871700D69797C50100B1
:1048700023ACE5D023807701630CC7047D1CE3C320
:1048800089FFB2476800A548B386F9008A061C086C
:10489000BE96294813030004370610F0E384A6E807
:1048A0009C429305000363F4F800930570051840DB
:1048B000AE9793051700569717CE01002326BECC5E
:1048C0002300F7006380072B638C6526F116F9B788
:1048D00017570300130707EB05078347F7FF23A0CC
:1048E000F6F01C40FD1797C5010023AFF5C8EDF7A2
:1048F0007D1C71B71C40130600041387170097C571
:10490000010023A3E5C8B386FA00930500032380C2
:10491000B6006300C73E890797C6010023A6F6C606
:104920005697930680072300D700175703001307F5
:1049300067E5B70610F0639EC70005078347F7FFDA
:1049400023A0F6F01C40FD1717C60100232EF6C267
:10495000EDF7A247C14C014D91072247014B832D32
:1049600007003EC455BDA24783AC0700138947002A
:10497000638F0C3A635480219307D002639EFB2E11
:1049800003C70C00BA856310072025AC8547A94CE6
:10499000014DE3C907E7A2479107C1B7A247834684
:1049A0001700528703AB070091073EC4E3580CDEA3
:1049B0005A8C7D5BE5B383461700930BD002528778
:1049C000F1BB9347FCFFFD8783461700337CFC0057
:1049D0005287E9B383461700930B000352877DBBD0
:1049E00003461700138B06FD5287930706FDB28618
:1049F000E3EEF8FA93172B00DA9705078607B297CC
:104A000003460700138B07FD930706FDB286E3F309
:104A1000F8FE69BFA2451C402946984193861700BD
:104A2000D69717C501002321D5B62380E700138947
:104A300045006301C72A930700046387F6204AC430
:104A4000D5B1854763DF0729A24713877700619BAC
:104A5000930787003EC4032B47001C43635B0B3066
:104A60001840130600049306170097C5010023ADF4
:104A7000D5B056979305D0022300B7006388C62CA3
:104A8000B307F0403337F000330B6041BE8D330B7A
:104A9000EB40A94C014D49B38346170005085287E6
:104AA000F5B9834617005287D5B91C409306000418
:104AB0001387170017C601002328E6ACD697130604
:104AC00050022380C700E31FD7C417570300130702
:104AD00067CBB70610F005078347F7FF23A0F6F072
:104AE0001C40FD1717C601002320F6AAEDF71DB9DB
:104AF000C14C014D29B31C40930600042A8A138738
:104B0000170017C601002321E6A8D6971306500206
:104B10002380C700E318D7C017570300130787C6C1
:104B2000B70610F005078347F7FF23A0F6F01C40F7
:104B3000FD1717C601002329F6A4EDF72A8ADDB672
:104B400017570300130707C405078347F7FF232000
:104B5000F6F01C40FD1797C5010023A7F5A2EDF75D
:104B6000F1162DBB175703001307C7C1F1FDF1164E
:104B700035B3E3FC9DCB8549C5B1014C03C70C009F
:104B8000BA85E30E07EAFD58294513080004B70665
:104B900010F063570B0A1C4013861700D69717C3F3
:104BA00001002323C39E2380E7006384A5066304DA
:104BB0000609850C03C70C007D1CBA8579FBE35000
:104BC00080E91C409305000213060004B70610F0AC
:104BD00021A07D1CE3050CE613871700D6972380E0
:104BE000B70017C501002321E59ABA87E313C7FE72
:104BF00017570300130707B905078347F7FF23A0DB
:104C0000F6F01C40FD1717C50100232FF596EDF7B0
:104C1000C9B7175703001307E7B641DE05078347F7
:104C2000F7FF23A0F6F01C40FD1717C60100232D47
:104C3000F694EDF7BDBF175703001307A7B4F9BFEC
:104C40007D1BE31A1BF5A5BF17570300130787B396
:104C5000B70610F005078347F7FF23A0F6F01C40C6
:104C6000FD1717C601002321F692EDF74AC45DBC7B
:104C700097BC0100938C0C75DA856685EF00707126
:104C8000330CAC40E35C80EF1C4013060004B70615
:104C900010F021A07D1CE3020CEE13871700D697BD
:104CA0002380770197C5010023A0E58EBA87E3131F
:104CB000C7FE175703001307E7AC05078347F7FF45
:104CC00023A0F6F01C40FD1797C5010023AEF58A1E
:104CD000EDF7C9B7175703001307C7AAB5FA4AC4B7
:104CE00091B4A247138747009C433AC413DBF741B2
:104CF000B5B3175703001307E7A8B70610F0050769
:104D00008347F7FF23A0F6F01C40FD1717C60100EC
:104D1000232CF686EDF7854717C701002326F78673
:104D20009307800717570300230EF7A41DB163569E
:104D300080019307D002E39DFBF297BC0100938CA6
:104D40006C68130780029305800235BD97560300F7
:104D5000938646A3370610F0850603C7F6FF232087
:104D6000E6F018407D1797C5010023AFE5806DF789
:104D700001BBBE8DA94C014D45B4B70710F023A06F
:104D8000A7F201A03971130341022ED29A8506CEF3
:104D900032D436D63AD83EDA42DC46DE1AC62D3256
:104DA000F2400145216182805D711303810322D4A9
:104DB0002AC632DC2A841A86680006D6BEC236DECF
:104DC000BAC0C2C4C6C61ACEEFF04FD4B2472380D1
:104DD00007003245B250018D225461618280B707CD
:104DE00010F083A647F403A607F403A747F4E31AD9
:104DF000D7FE856693868638B29633B6C600B3056D
:104E0000E60023A4D7F423A6B7F48280B70710F0F6
:104E100003A747F403A607F483A647F4E31AD7FED3
:104E2000856693868638B29633B6C60023A4D7F437
:104E3000B305E60023A6B7F49307000873A0473034
:104E40008280797122D406D626D24AD04ECE52CC58
:104E500056CA5AC85EC697B701009387677317B4DE
:104E600001001304A47298431C40930647069387DD
:104E7000470617B60100232BF670856717B60100A9
:104E80002328D670938777BB63CDD700B2502254C6
:104E900092540259F249624AD24A424BB24B45619E
:104EA0008280FD779387C74A3E9797B7010023A179
:104EB000E76E7D238547631DF504EF00D007854924
:104EC000114B814BA144314A814A2A89630335073A
:104ED00017B501001305C551EFF0DFEAEF00F03D13
:104EE000D2846306350717B501001305E552EFF0CC
:104EF0007FE92685EFF07FE82254B25092540259A0
:104F0000F249624AD24A424BB24B45616FC07FE8D8
:104F100017B501001305854BEFF0DFE6EF00B00198
:104F20008549194B894BA944394A894A2A89E31191
:104F300035FBEF009038E31825FB639C0A0018400E
:104F40008967938777328144E3C5E7FA81B7DA84CA
:104F50004DB7DE8479BF17B501001305254E6FF0FC
:104F60007FE217B501001305E54D6FF0BFE1411178
:104F700022C426C206C6856417B401001304044D7A
:104F8000938784380100FD17F5FF2285EFF09FDF3E
:104F9000C5BF411106C6A929D125B24041016F0004
:104FA0007027411106C622C426C25D2985476313B6
:104FB000F50491440144EF00007885476309F5004A
:104FC00017B501001305C542EFF0DFDB2684EF00C3
:104FD000D02E8547630AF50017B501001305C543B8
:104FE000EFF05FDA136484002285B24022449244D9
:104FF0004101828017B501001305453DEFF09FD8B0
:10500000994409444DBF7370043001A082807370CD
:10501000043001A0797126D24AD04ECE52CC56CA65
:105020005AC806D622D417BA0100130A6A5817BB09
:105030000100130B2B579304500505499309E00A0F
:10504000930AE00B0145EFD07F84EFC09FD62A84FE
:1050500003250A0081461306F00A6C0002C697B7C2
:10506000010023AD9752EFB00FF209C597B70100C9
:1050700023A82753EFC0FFD3018D63F4A90063F683
:10508000AA0097B7010023AD2751014597B701004A
:1050900023A69750EFD08FFFEFC0BFD12A840325FE
:1050A0000A0081461306F00A6C0097B7010023A797
:1050B000974EEFB07FBD09C597B7010023A2274FD8
:1050C000EFC03FCF018D63F4A90063F6AA0097B744
:1050D000010023A7274D97B7010023A1974C8327F1
:1050E0000B00850717B70100232EF74AA1BF3971BE
:1050F00026DA4AD84ED652D456D25AD05ECE62CC98
:1051000066CA06DE22DC6AC817BA0100130A4A4AD8
:1051100017B901001309894897BB0100938B0B490C
:1051200097BC0100938C4C48294C054B914A85490A
:105130009304500502C401463314CC00EFC07FC76E
:105140002A8D03250A00814622866C00EFB0DFB36A
:1051500009C597B7010023A53745EFC09FC53305A3
:10516000A5419307F4006376850017B70100232952
:10517000374363FDA724224697B7010023A2374394
:10518000050632C4E3DACAFA02C403250A008146DE
:1051900001462C00EFB02FDF6306652597B70100AD
:1051A00023A03741A24785073EC4E3D0FAFE02C4DC
:1051B00001463314CC00EFC0DFBF2A8D03250A005F
:1051C000814622862C00EFB00FDC09C597B701009D
:1051D00023A8373DEFC0FFBD3305A5419307F40079
:1051E0006376850017B70100232C373B63FAA71CB1
:1051F000224697B7010023A5373B050632C4E3DA00
:10520000CAFA03A50B0097B7010023A90738EFC01E
:10521000CFF983270900638997005145EFC0DFFB71
:1052200083270900E39B97FE5145EFC0FFFA97B72C
:10523000010023A5073602C403250A008146014662
:105240006C00EFB07FA4814601462C006306650127
:1052500097B7010023A6373503250A00EFB0AFD278
:1052600091456306650197B7010023AB3733832768
:10527000090003A50B006396970097B7010023A1CF
:105280003733EFC08FE083270900854503A50B0066
:105290006396970097B7010023A43731EFC0EFDE84
:1052A000A24785073EC4E3D9FAF883270900514590
:1052B00063899700EFC05FF2832709005145E39BA4
:1052C00097FEEFC07FF197B7010023A9072C02C416
:1052D00003250A00814601466C00EFB0FF9A630D7A
:1052E000650F97B7010023AD372BA24785073EC452
:1052F000E3D0FAFE03A50B00EFC02FEB83270900D4
:10530000638997005145EFC03FED83270900E39B78
:1053100097FE5145EFC05FEC97B7010023A0072827
:1053200002C403250A00814601462C00EFB0AFC538
:10533000814601466C006306650197B7010023A111
:10534000372703250A00EFB03F94914563066501B6
:1053500097B7010023A637258327090003A50B0073
:105360006396970097B7010023AC3723EFC0EFD1C6
:1053700083270900854503A50B006396970097B71F
:10538000010023AF3721EFC04FD0A24785073EC4AD
:10539000E3D9FAF883270900514563899700EFC0E4
:1053A000BFE3832709005145E39B97FEEFC0DFE28F
:1053B00083A70C00850717B701002327F71E9DBBA5
:1053C0002246050632C4E3D6CADE25BD22460506BE
:1053D00032C4E3D3CAD64DBBA24785073EC4E3D946
:1053E000FAEE09BFA24785073EC4E3D0FADAC1B39B
:1053F000411101469145154506C6EFB02FAC97B552
:1054000001009385E50597B7010023A3A71AEFB024
:105410001FCD814801488147094781461306004056
:1054200097B501009385050517050000130565CCA8
:10543000EFB05FEBB2408148014897B70100938716
:10544000E716054781461306004097B5010093858E
:10545000E50217050000130525BC41016FB09FE868
:1054600017B701001307471497B6010093868613F8
:1054700017B60100130606121C4310428C4217B5E2
:105480000100130565110328050001456386C50069
:10549000B38707413335F00097B701009387471072
:1054A0009C4394421843FD17B337F000B307F04014
:1054B00017B601002320D60E7D8D97B6010023ADCF
:1054C000E60C8280011122CC06CE26CA4AC84EC6FE
:1054D00052C458419307A00A2A8404416309F71073
:1054E0008146014681452685EFB00FFA8547631650
:1054F000F50097B7010023A3A70C05498549032AA6
:1055000004008146014681455285EFB0EFF7630400
:10551000250B9304800C8146014681455285EFB0EE
:105520008FA61C446300250D850717B701002327AC
:105530003709FD141CC4E5F08146014681455285BA
:10554000EFB06FA46316250197B7010023A82707C2
:10555000032A04008146014681455285EFB0AFA27F
:10556000630025079304800C8146014681455285DE
:10557000EFB08FF11C44630A2505850717B70100BA
:10558000232E3703FD141CC4E5F0814601468145F6
:105590005285EFB06FEFE31425F7032A040081462C
:1055A00001468145528597B7010023A92701EFB035
:1055B000AFEDE31025F797B7010023A1270191BFB5
:1055C00097B7010023AC27FF71BF8507FD141CC4EA
:1055D000C1FC8146014681455285EFB0EFEAE310F8
:1055E00025F365BF8507FD141CC495F4B1B781464A
:1055F000014681452685EFB00F9985476316F50072
:1056000097B7010023ACA7FA1309800C854981469E
:10561000014681452685EFB02FE71C44630A350318
:10562000850717B70100232B37F97D191CC4E31038
:1056300009FE2685814601468145EFB0EFE48547A6
:105640000440E31FF5E897B7010023A9A7F649BD79
:1056500085077D191CC4E31C09FAE1BF41119305BC
:10566000800C1305800C06C622C4EFB0AF8E97479E
:10567000030023A9A7149307A00A174703002325B3
:10568000F71481451305800C9747030023A00714E6
:10569000EFB04F8C9747030023ACA7129747030046
:1056A00023AA0712174403001304C41197470300E9
:1056B00023A40712084097B501009385A5DCEFB03D
:1056C0001FA2484497B501009385C5DCEFB03FA108
:1056D0001C40A1CF814801488147014797460300FC
:1056E0009386460E1306004097B50100938585DB2F
:1056F00017050000130545DDEFB0DFBE2244B240C0
:105700008148014881470147974603009386460C2C
:105710001306004097B50100938545D91705000091
:10572000130585DA41016FB0FFBB5C44C5F7B24099
:1057300022444101828017B70100130727E8104374
:10574000974703009387070817B701001307C7E6B9
:105750001843944701456389E600984713351600BE
:1057600097B6010023AAE6E417B70100130787E400
:10577000D44B18436388E600DC4B17B70100232B9A
:10578000F7E2828001458280797122D426D24AD004
:105790004ECE52CC56CA5AC85EC662C406D697B41C
:1057A00001009384A4E497B90100938969E217BAD0
:1057B0000100130AAAE197BA0100938A6AE297BB33
:1057C0000100938B2BE217BC0100130CACE00544E5
:1057D0000D49094B88408145EFB00FECE31C85FE75
:1057E00003A50900EFB0FFF7631C250B03250A0092
:1057F000EFB03FF76313250B83A70A006387870089
:1058000097B7010023A287DEF1B783A70B00E399C6
:1058100087FE83270C0003250A00850717B70100C0
:10582000232AF7DAEFC06F9803A50900EFC0EF97BE
:1058300083A70A006387870483A70B006383870419
:105840000145EFB05FFC6317650503A50900EFB0E4
:105850005FF1631D650503250A00EFB09FF0631437
:1058600065058840EFB00FA36306850097B7010078
:1058700023AC87D60145EFB01FF929DD73700430E2
:1058800001A0014597B7010023A087D6EFB0BFF76D
:10589000E30D65FB7370043001A07370043001A048
:1058A0007370043001A07370043001A07370043071
:1058B00001A0011122CC26CA4AC84EC652C406CE47
:1058C00017B90100130989D217BA0100130A8AD146
:1058D00097B40100938444D097B90100938909D00B
:1058E00005442DA097B7010023A087D09C4003A7B3
:1058F000090085076386E70097B7010023A687CED6
:105900009C40850717B701002328F7CC0325090021
:10591000F955EFB06FD8E31785FC83270A00E393AE
:1059200087FC03250900EFB0EF966306850097B763
:10593000010023AB87CA014597B7010023A287CA9C
:10594000EFC0DFF497B7010023AC07C845B70111DA
:105950004AC817B90100130969C90325090022CCF7
:105960004EC606CE26CA054497B90100938909C7D9
:10597000EFB04F9263058508A94403250900A145AE
:10598000EFB08FD163028508FD14514597B7010030
:1059900023AC87C4EFC05F84EDF0A9445145EFC04C
:1059A000BF8303250900FD14EFB0CF8E6306850089
:1059B00097B7010023AA87C2F5F003250900EFB0CD
:1059C0006F8D6316850097B7010023AF87C083A74B
:1059D00009000145850717B701002321F7C097B7D4
:1059E000010023A187C0EFC07FEA0325090097B714
:1059F000010023A907BEEFB0EF89E31F85F697B733
:105A0000010023A387BE8DBFFD145145EFC0CFFC1D
:105A1000ADF461B74111114506C6EFB0EF8197B5FE
:105A20000100938525A997B7010023A1A7BCEFB07A
:105A30000FEB97B70100938767BB9C43A5CF8148C5
:105A4000014897B701009387A7B809478146130615
:105A5000004097B501009385E5A6170500001305E2
:105A600045EFEFB03F888148014897B70100938721
:105A7000E7B5054781461306004097B501009385B9
:105A8000E5A417050000130505E3EFB0BF85B2409C
:105A9000814801488147014781461306004097B578
:105AA0000100938525A317050000130525CE4101AC
:105AB0006FB05F83B2404101828097B70100938746
:105AC000E7B197B60100938626B09843944263826B
:105AD000E6069C4397B601009386C6AE944217B77C
:105AE00001002323F7AE97B701009387E7AE9843F1
:105AF0006382E6069C4397B60100938666AC9442A7
:105B000017B701002320F7AC97B70100938787AC44
:105B100098436382E6069C4317B701002322F7AA45
:105B200097B70100938747AC88437D153335A000B4
:105B30008280854717B701002328F7AA97B601008E
:105B4000938646A897B70100938707A99843944284
:105B5000E392E6FA854717B701002327F7A897B61F
:105B600001009386E6A597B701009387A7A69843FF
:105B70009442E392E6FA854717B701002326F7A679
:105B800097B70100938747A688437D153335A0005A
:105B90008280AA95AA876385B70003C7070001E73B
:105BA0003385A74082808507FDB7814863DA050009
:105BB0003305A040B337A000B305B0409D8DFD581C
:105BC00063D906003306C040B337C000B306D040E7
:105BD0009D8E32883683AA872E87639F061C97A6E0
:105BE00001009386266D63F1C50C416E6377C60B89
:105BF000130EF00F6373CE002143335E6600F296FE
:105C000003CE06001A9E130300023303C341630C44
:105C10000300B3956500335EC50133186600336732
:105C2000BE00B3176500135E0801B355C703131513
:105C30000801418193D607013376C703B305B50246
:105C40004206D18E63F8B600C29663E5060163F39F
:105C5000B600C2968D8E33F7C603C207C183B3D692
:105C6000C603B306D50213150701C98F63F8D70021
:105C7000C29763E5070163F3D700C297958F33D5C9
:105C800067008145638A0800B307A0403337F000FE
:105C9000B305B0403E85998D8280370E00014143A7
:105CA000E36DC6F5614391BF01E6054833586802CC
:105CB00041676373E8081307F00F6373070121431B
:105CC00033576800BA9603C606001A9613030002FB
:105CD0003303C34063190306B38505419356080196
:105CE00013150801418113D6070133F7D502B3D547
:105CF000D5024207518FB305B5026378B7004297CA
:105D0000636507016373B7004297B305B74033F784
:105D1000D502C207C183B3D5D502B305B5021315A9
:105D20000701C98F63F8B700C29763E5070163F302
:105D3000B700C2978D8FA1B7370700014143E361D8
:105D4000E8F86143B5BF3318680033DEC500935EE1
:105D500008013356C500B31765003355DE03B3950C
:105D600065004D8E93150801C18193560601337766
:105D7000DE033385A5024207558F6378A70042975B
:105D8000636507016373A7004297B306A74033F723
:105D9000D60342064182B3D6D6034207B386D50264
:105DA000B365C70063F8D500C29563E5050163F3E9
:105DB000D500C295958D1DB7E3E6D5EC416863F536
:105DC0000605930EF00F33B8DE000E0833DE060131
:105DD00017A301001303034E7293834E0300130EA7
:105DE0000002C29E330EDE4163170E0263E4B6006A
:105DF0006369C500B307C540958D3335F50033871A
:105E0000A5403E85BA85BDBD370300014148E3EF9B
:105E100066FA614865BF3357D601B396C601D98E7D
:105E2000B357D50133D7D501B395C501CD8F93D5E0
:105E300006013373B702139F0601135F0F0113D8D6
:105E400007013316C6013315C5013357B7024203A4
:105E500033680301B30FEF023A83637CF80136988D
:105E60001303F7FF6367D8006375F8011303E7FFB7
:105E700036983308F841B37FB8023358B802C20FDE
:105E8000B3050F03139F0701135F0F0133EFEF01FA
:105E90004287637CBF00369F1307F8FF6367DF000C
:105EA0006375BF001307E8FF369F4203C16F33637A
:105EB000E3009387FFFF13580601330FBF40B3750C
:105EC000F30013530301F18F3387F502B307F30295
:105ED000B385050333030303BE95135807012E98BA
:105EE0006373F8007E93C167FD17935508013378FB
:105EF000F80042087D8F9A9542976366BF00631B46
:105F0000BF006379E5003306C7403337C700958D7E
:105F1000998D32873307E5403335E500B305BF403F
:105F2000898DB397D5013357C70133E5E700B3D562
:105F3000C50189BBAE87328836872A8363960620DF
:105F400097A801009388083763FEC50A4167637408
:105F5000E60A1307F00F3337C7000E07B356E60003
:105F6000B69883C60800369793060002998E99CAA0
:105F7000B397D7003357E5003318D600B365F70061
:105F80003313D50013550801B3D7A5021316080122
:105F900041829356030133F7A502B305F602420787
:105FA000D98E3E8763FCB600C2961387F7FF63E77E
:105FB000060163F5B6001387E7FFC2968D8EB3F72F
:105FC000A602420313530301B3D6A602C20733E36A
:105FD0006700B305D6023685637BB3004293138511
:105FE000F6FF636603016374B3001385E6FF42079F
:105FF000498F81454DA8B70600014147E360D6F6B9
:106000006147A9BF01E6854633D8C602C166637EF3
:10601000D8089306F00F63F306012147B356E80052
:10602000B69883C60800BA9613070002158F49E791
:10603000B38707418545135608019318080193D883
:1060400008019356030133F7C702B3D7C7024207CB
:10605000D98E3385F8023E8763FCA600C29613876B
:10606000F7FF63E7060163F5A6001387E7FFC29613
:10607000898EB3F7C602420313530301B3D6C60297
:10608000C20733E36700B388D8023685637B130108
:1060900042931385F6FF636603016374130113854E
:1060A000E6FF4207498F3A858280B70600014147E3
:1060B000E366D8F661479DB73318E800B3D5D7003B
:1060C0003313E500B356D50013550801B397E70025
:1060D00033F7A502B3E8F60093170801C18313D67E
:1060E0000801B3D5A5024207518FB386B7022E86A9
:1060F000637CD70042971386F5FF636707016375DA
:10610000D7001386E5FF4297B306D74033F7A602C0
:10611000C20893D80801B3D6A6024207B385D702B6
:10612000B3671701368763FCB700C2971387F6FF82
:1061300063E7070163F5B7001387E6FFC2978D8F0A
:1061400093150601D98DC5BD63E2D514416763FE81
:10615000E6021308F00F3337D8000E0733D8E600F5
:1061600097A5010093850515C29503C80500930501
:1061700000023A98B385054185E10547E3E5F6F26B
:106180003335C5001347150039BFB7050001414736
:10619000E3E6B6FC6147D9B733570601B396B600BC
:1061A000D98E93DE060133D70701B378D703B397AF
:1061B000B700335805013363F80093970601C18394
:1061C000135803013316B6003357D703C20833E818
:1061D0000801338FE7023A8E637CE8013698130E8C
:1061E000F7FF6367D8006375E801130EE7FF369881
:1061F0003308E841B378D8033358D803C208B38EC4
:10620000070393170301C183B3E7F800428763FCD8
:10621000D701B6971307F8FF63E7D70063F5D701F7
:106220001307E8FFB697420EB387D741C16E3367B5
:10623000EE001388FEFF337307019358070133788C
:1062400006014182330E03033388080393560E017F
:106250003303C30242939A96B388C80263F30601DC
:10626000F69813D60601B29863E01703E39317D9A3
:10627000C167FD17FD8EC206337EFE003315B500E3
:10628000F2968145E371D5E27D17A5B381450147BB
:1062900019BDB2883687AA872E886398061C97A6F0
:1062A00001009386260163F8C50A4163637E660890
:1062B0001303F00F6373C30021473353E6009A962C
:1062C00003CE0600130300023A9E3303C341630C5E
:1062D0000300B3956500335EC501B31866003368EB
:1062E000BE00B317650013D608013377C8021395B3
:1062F0000801418193D607013358C8024207D98E5D
:106300003308050363F80601C69663E5160163F3D7
:106310000601C696B386064133F7C602C207C1839B
:10632000B3D6C602B306D50213150701C98F63F8A9
:10633000D700C69763E5170163F3D700C697958F1B
:1063400033D5670081458280370300014147E3660A
:1063500066F661479DB701E60546B35816034166E8
:1063600063F3C8081306F00F63731601214733D691
:10637000E800B29603CE0600130300023A9E3303F0
:10638000C34163190306B385154113D7080113955B
:106390000801418113D60701B3F6E502B3D5E50242
:1063A000C206D18EB305B50263F8B600C69663E5A2
:1063B000160163F3B600C696B385B640B3F6E502A0
:1063C000C207C183B3D5E502B305B5021395060133
:1063D000C98F63F8B700C69763E5170163F3B70089
:1063E000C6978D8FB1BF370600014147E3E1C8F87A
:1063F0006147B5BFB398680033D7C501B3176500CF
:10640000335EC50113D50801B376A702B3956500C5
:10641000336EBE0093950801C18113560E013357A8
:10642000A702C206D18E3387E50263F8E600C6965E
:1064300063E5160163F3E600C6963386E640B3765D
:10644000A602420E135E0E013356A602C206338622
:10645000C502B3E5C60163F8C500C69563E515013D
:1064600063F3C500C695918D0DB7E3EED5EC41679A
:1064700063F5E604930EF00F33B7DE000E0733D357
:10648000E60097A801009388E8E29A9883CE080076
:10649000130E0002BA9E330EDE4163170E0263E450
:1064A000B6006369C500B307C540958D3335F50067
:1064B0003388A5403E85C28579B5B70800014147BC
:1064C000E3EF16FB614765BF3357D601B396C601AC
:1064D000D98EB357D50133D7D501B395C501CD8F2B
:1064E00093D506013373B702139F0601135F0F01A3
:1064F00093D807013316C6013315C5013357B702C8
:106500004203B36813013308EF023A8363FC0801C6
:10651000B6981303F7FF63E7D80063F50801130388
:10652000E7FFB698B3880841B3FFB802B3D8B80202
:10653000C20FB3051F03139F0701135F0F0133EF52
:10654000EF014687637CBF00369F1387F8FF6367C0
:10655000DF006375BF001387E8FF369F4203C16801
:106560003363E3009387F8FF13580601330FBF40EE
:10657000B375F30013530301F18F3387F502B307AB
:10658000F302B385050333030303BE9513580701D4
:106590002E986373F8004693C167FD179355080161
:1065A0003378F80042087D8F9A9542976366BF0062
:1065B000631BBF006379E5003306C7403337C7006C
:1065C000958D998D32873307E5403335E500B30566
:1065D000BF40898DB397D5013357C70133E5E70035
:1065E000B3D5C5018DB3011122CC26CA2A84AE844D
:1065F0004AC84EC652C456C206CEEFB08FFA1C40EF
:1066000003290401B7090001B3E59700930AC40008
:106610000CC08144FD19370A00021840638C2A031C
:10662000032609004A85B3654701B37636019317FF
:106630005600758F0329490063C4070001E7F1BFC5
:10664000E39DE6FC9317760063D30700D58CEFC07B
:106650006FE2E1B793C4F4FFF98C04C0EFB07F9907
:106660000840F2406244D2444249B249224A924A26
:1066700005618280411106C622C4EFE07FD7EFE0BA
:10668000FFFDEFF02FB917E7FFFF1307C77B814628
:1066900005469305400617A501001305A5DBEFD0BD
:1066A0006FB119C92A84EFB0CFF02A86014781461D
:1066B00085452285EFD0AFBCEFB08FC7B2402244F2
:0666C0000145410182804A
:02000004800278
:100000003E45FEFF3C46FEFF4645FEFF3C46FEFFEA
:100010003C46FEFF3C46FEFF3C46FEFF5E45FEFFC3
:100020003C46FEFF3C46FEFF7845FEFF8445FEFF52
:100030003C46FEFF9645FEFFA245FEFFA245FEFFA1
:10004000A245FEFFA245FEFFA245FEFFA245FEFF20
:10005000A245FEFFA245FEFFA245FEFF3C46FEFF75
:100060003C46FEFF3C46FEFF3C46FEFF3C46FEFF94
:100070003C46FEFF3C46FEFF3C46FEFF3C46FEFF84
:100080003C46FEFF3C46FEFF3C46FEFF3C46FEFF74
:100090003C46FEFF3C46FEFF3C46FEFF3C46FEFF64
:1000A0003C46FEFF3C46FEFF3C46FEFF3C46FEFF54
:1000B0003C46FEFF3C46FEFF3C46FEFF3C46FEFF44
:1000C0003C46FEFF3C46FEFF3C46FEFF3C46FEFF34
:1000D0003C46FEFF3C46FEFF3C46FEFF3C46FEFF24
:1000E0003C46FEFF3C46FEFF3C46FEFF3C46FEFF14
:1000F0003C46FEFF3C46FEFF3C46FEFF3C46FEFF04
:10010000D645FEFFEC45FEFF3C46FEFF3C46FEFFAB
:100110003C46FEFF3C46FEFF3C46FEFF3C46FEFFE3
:100120003C46FEFF3246FEFF3C46FEFF3C46FEFFDD
:10013000E443FEFF9C44FEFF3C46FEFF3C46FEFFC0
:10014000D244FEFF3C46FEFF2A45FEFF3C46FEFF32
:100150003C46FEFF5845FEFF4A49FEFF9E49FEFF12
:100160005249FEFF9E49FEFF9E49FEFF9E49FEFF4B
:100170009E49FEFF4448FEFF9E49FEFF9E49FEFF4A
:100180005E48FEFF6A48FEFF9E49FEFF7C48FEFF78
:100190008848FEFF8848FEFF8848FEFF8848FEFF2B
:1001A0008848FEFF8848FEFF8848FEFF8848FEFF1B
:1001B0008848FEFF9E49FEFF9E49FEFF9E49FEFFC6
:1001C0009E49FEFF9E49FEFF9E49FEFF9E49FEFF9F
:1001D0009E49FEFF9E49FEFF9E49FEFF9E49FEFF8F
:1001E0009E49FEFF9E49FEFF9E49FEFF9E49FEFF7F
:1001F0009E49FEFF9E49FEFF9E49FEFF9E49FEFF6F
:100200009E49FEFF9E49FEFF9E49FEFF9E49FEFF5E
:100210009E49FEFF9E49FEFF9E49FEFF9E49FEFF4E
:100220009E49FEFF9E49FEFF9E49FEFF9E49FEFF3E
:100230009E49FEFF9E49FEFF9E49FEFF9E49FEFF2E
:100240009E49FEFF9E49FEFF9E49FEFF9E49FEFF1E
:100250009E49FEFF9E49FEFFBC48FEFFEA48FEFFA6
:100260009E49FEFF9E49FEFF9E49FEFF9E49FEFFFE
:100270009E49FEFF9E49FEFF9E49FEFF4049FEFF4C
:100280009E49FEFF9E49FEFFA246FEFF9C47FEFFE1
:100290009E49FEFF9E49FEFF0E48FEFF9E49FEFF5F
:1002A0003448FEFF9E49FEFF9E49FEFF9849FEFF2F
:1002B000000102020303030304040404040404040D
:1002C00005050505050505050505050505050505DE
:1002D00006060606060606060606060606060606BE
:1002E00006060606060606060606060606060606AE
:1002F000070707070707070707070707070707078E
:10030000070707070707070707070707070707077D
:10031000070707070707070707070707070707076D
:10032000070707070707070707070707070707075D
:10033000080808080808080808080808080808083D
:10034000080808080808080808080808080808082D
:10035000080808080808080808080808080808081D
:10036000080808080808080808080808080808080D
:1003700008080808080808080808080808080808FD
:1003800008080808080808080808080808080808ED
:1003900008080808080808080808080808080808DD
:1003A00008080808080808080808080808080808CD
:1003B000546D725100000000546D7220537663003A
:1003C000286E756C6C2900004572726F7220696E20
:1003D00020626C6F636B2074696D65207465737443
:1003E000207461736B73200D0A0000004572726FF8
:1003F0007220696E20636F756E74696E6720736515
:100400006D6170686F7265207461736B73200D0A83
:10041000000000004572726F7220696E2072656381
:10042000757273697665206D757465782074617373
:100430006B73200D0A0000006D69616F750A000082
:100440006D69616F75320A0068756E6772790A00AE
:10045000436865636B54696D65720000426C6F633D
:100460006B5F54696D655F517565756500000000CF
:100470004254657374310000425465737432000055
:10048000436F756E74696E675F53656D5F31000011
:10049000436F756E74696E675F53656D5F32000000
:1004A000434E543100000000434E5432000000001F
:1004B0005265637572736976655F4D757465780012
:1004C0005265633100000000526563320000000095
:0804D0005265633300000000D7
:1004D8001000000000000000017A5200017C0101B8
:1004E8001B0D02001000000018000000B656FEFFA9
:1004F8008A03000000000000100000002C0000002B
:100508002C5AFEFF5E0300000000000010000000EF
:1005180040000000765DFEFF54030000000000006C
:0805EC00FC8F01000400000077
:040000058000004037
:00000001FF
